:100000000C9487060C94A4060C94A4060C94A406E5
:100010000C94A4060C94A4060C94A4060C94A406B8
:100020000C94A4060C94A4060C94A4060C94A406A8
:100030000C94A4060C94A4060C94A4060C94A40698
:100040000C94A4060C94A4060C94A4060C94A40688
:100050000C94A4060C94A4060C94A4060C94A40678
:100060000C94A4060C94A4060C94A4060C94A40668
:100070000A507265706172696E6720746F207072C9
:100080006F6772616D2041746D656C20323035315F
:100090002F343035312E2E2E00204F4B2E0056653A
:1000A00072696669636174696F6E204661696C6527
:1000B0006421002E000A566572696679696E6720B0
:1000C00070726F6772616D20646174612E2E2E00F4
:1000D0000A000A556E6B6E6F776E20506172742E37
:1000E0002E2E436865636B20436F6E6E6563746983
:1000F0006F6E73002E2041746D656C203430353185
:100100002E20002E2041746D656C20323035312E4A
:100110002000203078003078000A44657465726DE4
:10012000696E696E67206368697020747970652EE6
:100130002E2E004F4B2E000A436C656172696E676C
:1001400020636869702E2E2E2000204F4B2E200039
:100150002E000A57726974696E6720636869702E91
:100160002E2E000A53696D706C7920636C65617284
:10017000206F7220726570726F6772616D20746893
:10018000652047414C20746F20636C656172207458
:100190006865207365637572697479206675736527
:1001A000000A77696C6C2067697665206120766546
:1001B00072696669636174696F6E206572726F72CD
:1001C0002061667465722070726F6772616D6D690F
:1001D0006E672E000A4265636175736520746869F5
:1001E000732077696C6C2070726576656E7420720E
:1001F000656164696E67206F757420746865206638
:10020000757365206D61702C207468697320474197
:100210004C000A596F7520686176652063686F73BA
:10022000656E20746F2070726F6772616D207468E4
:10023000652053656375726974792046757365200E
:10024000696E2074686973204A454445432E000A4C
:10025000436865636B73756D2057726F6E67000A34
:100260004E6F204675736520436865636B73756DCB
:100270002070726573656E7420696E204A4544452E
:10028000432066696C652E2020436865636B20639C
:100290006F6D70696C65722073657474696E6773D5
:1002A000000A54686973204A4544454320686173D5
:1002B000207468652077726F6E67206E756D626559
:1002C00072206F662070696E73206F72206E6F20CF
:1002D00070696E206465636C61726174696F6E2E03
:1002E0002020497320697420666F72206120474185
:1002F0004C32325631303F000A54686973204A4507
:1003000044454320686173207468652077726F6E7E
:1003100067206E756D626572206F66206675736505
:1003200073206F72206E6F2066757365206465633D
:100330006C61726174696F6E2E202049732069743C
:1003400020666F7220612047414C32325631303F77
:10035000002E000A3E000A000A696E76616C69642C
:1003600020636F6D6D616E64000A56202020205658
:100370006965772074686520636F6465206F6E20FF
:100380007468652063757272656E746C7920696E2D
:1003900073657274656420323035312F34303531F5
:1003A0002E000A48202020205072696E7420746844
:1003B00069732068656C7020646F63756D656E7419
:1003C0002E000A41202020204175746F20446F7751
:1003D0006E6C6F616420616E642050726F67726131
:1003E0006D20323035312F343035312E000A442023
:1003F000202020446F776E6C6F616420616E20490D
:100400006E74656C204865782066696C6520746F31
:10041000204255524E49542E000A432020202043AA
:100420006C65617220616E2041544D454C20323024
:1004300035312F343035312E000A50202020205005
:10044000726F6772616D20616E2041544D454C2082
:10045000323035312F343035312E000A4255524E6C
:1004600049542048656C70000A696E76616C696455
:1004700020636F6D6D616E64000A4820202020505B
:1004800072696E7420746869732068656C7020648A
:100490006F63756D656E742E000A562020202056FD
:1004A00069657720467573656D6170206F66206998
:1004B0006E7365727465642047414C2E000A4120BA
:1004C0002020204175746F20446F776E6C6F6164DB
:1004D00020616E642050726F6772616D20612047E9
:1004E000414C2E000A4420202020446F776E6C6F10
:1004F00061642061204A454445432066696C65205B
:10050000746F204255524E49542E000A4320202039
:1005100020436C65617220612047414C2E000A50D7
:100520002020202050726F6772616D20612047414A
:100530004C2E000A4255524E49542048656C7000BA
:100540000A566572696669636174696F6E204F4B04
:100550002E000A566572696669636174696F6E2060
:100560004572726F72000A47414C2050726F677279
:10057000616D6D65642E2E2E566572696679696EA1
:10058000672E2E2E000A50726F6772616D6D696E54
:10059000672047414C2E2E2E000A47414C204572C1
:1005A00061736564000A45726173696E6720474133
:1005B0004C2E2E2E000A4552524F5220696E206456
:1005C0006F776E6C6F6164696E67204A454445437E
:1005D0002E2E2E4175746F70726F6772616D6D692A
:1005E0006E672077696C6C206E6F7420636F6E7419
:1005F000696E7565000A4A4544454320446F776E2D
:100600006C6F616420436F6D706C657465000A45A2
:1006100052524F5220696E20646F776E6C6F616426
:10062000696E67204A45444543000A4A45444543AC
:1006300020446F776E6C6F616420436F6D706C65E2
:100640007465000A47414C20457261736564000A75
:1006500045726173696E672047414C2E2E2E000A49
:10066000696E76616C696420636F6D6D616E6400A4
:100670000A5520202020556E6C6F636B2050494333
:1006800020696620636F64652070726F746563749F
:10069000696F6E20656E61626C65642E000A56207B
:1006A000202020566965772074686520636F646533
:1006B000206F6E207468652063757272656E746C4D
:1006C0007920696E736572746564205049432E0009
:1006D0000A48202020205072696E74207468697363
:1006E0002068656C7020646F63756D656E742E0094
:1006F0000A41202020204175746F20446F776E6C72
:100700006F616420616E642050726F6772616D204A
:100710005049432E000A4420202020446F776E6CFD
:100720006F616420616E20496E74656C2048657845
:100730002066696C6520746F204255524E49542ED4
:10074000000A4320202020436C6561722061205004
:1007500049432E000A502020202050726F6772619A
:100760006D2061205049432E000A4255524E495493
:100770002048656C70000A4255524E49543E000AAA
:1007800047414C3232563130206D6F646520656EC2
:1007900061626C6564000A41746D656C20323035AD
:1007A00031206D6F646520656E61626C6564000A5E
:1007B000506C6561736520636F727265637420614C
:1007C0006E64207265736574204275726E49740A96
:1007D000000A4D61796265207468652063686970FC
:1007E0002069736E277420696E7365727465642066
:1007F0006F72207468652073776974636820697309
:1008000020696E207468652077726F6E6720706F44
:10081000736974696F6E2E000A504943206D6F64CE
:100820006520656E61626C6564000A57656C636F74
:100830006D6520746F204255524E4954210A507202
:100840006573732027482720666F722068656C7077
:100850002E002E000A4552524F523A2043686563DB
:100860006B73756D20696E76616C696420696E20AA
:100870006865782066696C652E000A436865636B5D
:1008800020796F757220636F6D70696C657220736B
:10089000657474696E6773206F7220676574206178
:1008A000203136463632382E000A4552524F523ADF
:1008B0002054686973206865782066696C652068D3
:1008C0006173206D6F72652064617461207468616A
:1008D0006E207468652050494331364636323720E1
:1008E00063616E20686F6C642E00746F20446174C5
:1008F00061206F7220436F6E666967206D656D6F52
:1009000072792E20204974206D6967687420616CAB
:10091000736F20626520746F6F2062696720666F55
:1009200072207468697320636869702E000A4552EA
:10093000524F523A2054686973206865782066697E
:100940006C6520686173206461746120696E206841
:10095000696768206D656D6F7279207468617420B5
:10096000646F6573206E6F7420636F72726573704D
:100970006F6E640A000A5761726E696E673A206989
:10098000676E6F72696E6720484558207265636FA5
:10099000726420000A3E000A506572666F726D69CB
:1009A0006E6720746F74616C2062756C6B20657269
:1009B00061736520746F20636C65617220636F647E
:1009C000652070726F74656374696F6E2E2E2E00D1
:1009D0000A20434F4E46494720574F5244203A2061
:1009E000000A2055534552204944203A20000A006D
:1009F0000A2044415441203A000A000A556E6B6EA9
:100A00006F776E205049432C20436F6E66696720D4
:100A1000776F7264207761733A000A504943313628
:100A200046363238206465746563746564000A5024
:100A300049433136463632372064657465637465E0
:100A400064000A50494331364636323841206465E5
:100A5000746563746564000A504943313646363222
:100A60003741206465746563746564000A497420C5
:100A700063616E20616C736F206F6E6C7920707291
:100A80006F6772616D207468652066697273742087
:100A9000313238206279746573206F662044617446
:100AA0006120616E64206E6F7420616C6C20323541
:100AB000362062797465732E000A344B206F6620ED
:100AC0006D656D6F7279206F6E2074686973206434
:100AD00065766963652E000A4E6F74653A20546826
:100AE00069732070726F6772616D6D6572206361EA
:100AF0006E206F6E6C792070726F6772616D2074FA
:100B0000686520666972737420324B206F66206DB1
:100B1000656D6F727920616E64206E6F74207468E9
:100B2000652077686F6C65000A5049433136463658
:100B300034384120646574656374656400496620D7
:100B4000746861742077617320746865206F6E6CBF
:100B5000792070726F626C656D2C20646F206E6FEF
:100B60007420776F7272792E000A4E4F54453A20E6
:100B7000546869732070726F6772616D6D65722061
:100B800063616E6E6F742064697361626C65204C82
:100B90006F7720566F6C746167652050726F677253
:100BA000616D6D696E670A000A20526561643A20C2
:100BB000000A2053656E743A20000A566572696611
:100BC00069636174696F6E206572726F72206475FB
:100BD00072696E6720436F6E6669677572617469CA
:100BE0006F6E2070726F6772616D6D696E672E0037
:100BF0000A50726F6772616D6D696E67205049436C
:100C000020436F6E66696775726174696F6E2057F5
:100C10006F72642E2E2E000A5665726966696361D2
:100C200074696F6E206572726F7220647572696E7E
:100C30006720446174612070726F6772616D6D69C5
:100C40006E672E000A50726F6772616D6D696E6714
:100C5000205049432044617461206D656D6F727945
:100C60002E2E2E000A436F64652070726F746563C8
:100C700074696F6E206D617920626520656E6162B6
:100C80006C65642E000A56657269666963617469F1
:100C90006F6E206572726F7220647572696E672064
:100CA00070726F6772616D6D696E672E002E000A3B
:100CB00050726F6772616D6D696E67205049432095
:100CC00050726F6772616D206D656D6F72792E2E37
:100CD0002E000A45726173696E6720504943206493
:100CE000617461206D656D6F72792E2E2E000A453C
:100CF000726173696E67205049432070726F67722A
:100D0000616D206D656D6F72792E2E2E000011249D
:100D10001FBECFEFD0E1DEBFCDBF13E0A0E0B1E05A
:100D2000E4EEF7E702C005900D92A232B107D9F7C1
:100D30001EE0A2E2B3E001C01D92A73AB107E1F7BD
:100D40000E94E6190C94F03B0C9400002F9A82E06C
:100D5000982F9A95F1F72F988A95F1F708950F93A8
:100D60001F93CF93DF9385EB90E00E946E0911B83B
:100D700015B88AE18A95F1F785B1816485B985B1A5
:100D80008F7C85B985B18C6085B985E08A95F1F74E
:100D9000C0E0D0E012E005E017C080B1FE01E55FE1
:100DA000F94F9081981701F52F9A812F8A95F1F7C5
:100DB0002F98812F8A95F1F7802F8A95F1F7219648
:100DC00088E0C030D807E9F0CE018F779070892B8A
:100DD00021F783EB90E00E946E0980B1FE01E55F90
:100DE000F94F9081981701F38EE990E00E946E0907
:100DF00015B88FEF81B912B8DF91CF911F910F9184
:100E0000089515B88FEF81B912B889E990E00E9472
:100E10006E09DF91CF911F910F91089587E391E0C3
:100E20000E946E0915B885B1816485B92D9A85B186
:100E3000837E85B98AE18A95F1F7299A80E28A95BD
:100E4000F1F72E9880E29EE4FC013197F1F72E9A9B
:100E5000FC013197F1F729980197F1F715B883E371
:100E600091E00E946E090895FF920F931F93CF9314
:100E7000DF9382E591E00E946E0915B812B88AE10D
:100E80008A95F1F785B1816485B92D9885B18C611A
:100E900085B985E08A95F1F7299A80E58A95F1F779
:100EA000C0E0D0E005E08AE1F82E12E0CE018F77B5
:100EB0009070892B09F435C0FE01E55FF94F808100
:100EC00082B9802F8A95F1F72E988F2D8A95F1F7A8
:100ED0002E9A3099FECF309BFECF2F9A812F8A9584
:100EE000F1F72F98812F8A95F1F7802F8A95F1F7E6
:100EF000219688E0C030D807C9F680E29EE4FC0164
:100F00003197F1F729980197F1F715B812B88AE4EB
:100F100091E00E946E09DF91CF911F910F91FF9098
:100F2000089580E591E00E946E09C6CFAF92BF920E
:100F3000CF92DF92EF92FF920F931F93DF93CF93A5
:100F4000CDB7DEB72A970FB6F894DEBF0FBECDBF80
:100F500011B815B88AE18A95F1F785B1816485B930
:100F600085B18F7C85B985B18C6085B985E08A951E
:100F7000F1F700E010E030E0A32E31E0B32E6E0177
:100F80000894C11CD11C22E0F22E95E0E92E14C079
:100F900080B10E948D092F9A8F2D8A95F1F72F9895
:100FA0008F2D8A95F1F78E2D8A95F1F70F5F1F4FE0
:100FB00098E000301907E9F0C8018F719070892B13
:100FC00039F780ED90E00E946E091F930F93BF9256
:100FD000AF92DF92CF920E94DD38C6010E94550980
:100FE0008DB79EB706960FB6F8949EBF0FBE8DBF05
:100FF000CFCF15B88FEF81B912B82A960FB6F894F3
:10100000DEBF0FBECDBFCF91DF911F910F91FF903B
:10101000EF90DF90CF90BF90AF9008950F931F9304
:1010200089E191E00E946E0911B815B88AE18A95AC
:10103000F1F785B1816485B985B1837C85B986E195
:1010400091E00E946E0915E0812F8A95F1F700B1B9
:10105000802F0E948D0982E191E00E946E092F9AF3
:1010600082E0982F9A95F1F72F988A95F1F71A95C3
:10107000F1F710B1812F0E948D0915B88FEF81B95A
:1010800012B80E3151F082ED90E00E946E0921E01D
:1010900030E0C9011F910F910895113249F01134C8
:1010A00091F784EF90E00E946E0920E030E0F1CFEC
:1010B00083E091E00E946E0920E030E0EACFFF92E9
:1010C0000F931F93CF93DF9380E790E00E946E0908
:1010D0000E940E08892B31F0DF91CF911F910F9163
:1010E000FF90089587E391E00E946E0915B885B1DD
:1010F000816485B92D9A85B1837E85B91AE1812FE6
:101100008A95F1F7299A80E28A95F1F72E9880E284
:101110009EE4FC013197F1F72E9AFC013197F1F72B
:1011200029980197F1F715B883E391E00E946E09C1
:1011300082E591E00E946E0915B812B81A95F1F790
:1011400085B1816485B92D9885B18C6185B985E0BB
:101150008A95F1F7299A80E58A95F1F7C0E0D0E009
:1011600005E04AE1F42E12E0CE018F779070892BD2
:1011700009F47EC0FE01E55FF94F808182B9802FBE
:101180008A95F1F72E988F2D8A95F1F72E9A30993E
:10119000FECF309BFECF2F9A812F8A95F1F72F98A3
:1011A000812F8A95F1F7802F8A95F1F7219688E0B3
:1011B000C030D807C9F680E29EE4FC013197F1F710
:1011C00029980197F1F715B812B88AE491E00E94C6
:1011D0006E0985EB90E00E946E0911B815B88AE19E
:1011E0008A95F1F785B1816485B985B18F7C85B920
:1011F00085B18C6085B985E08A95F1F7C0E0D0E0D3
:1012000012E005E017C080B1FE01E55FF94F908163
:10121000891701F52F9A812F8A95F1F72F98812F41
:101220008A95F1F7802F8A95F1F7219688E0C030F2
:10123000D80719F1CE018F779070892B21F783EBB6
:1012400090E00E946E0980B1FE01E55FF94F908148
:10125000891701F38EE990E00E946E0915B88FEFAF
:1012600081B912B8DF91CF911F910F91FF9008952E
:1012700080E591E00E946E097DCF15B88FEF81B9AE
:1012800012B889E990E00E946E0926CF982F8091CC
:10129000C00085FFFCCF9093C60008958091C000E8
:1012A00087FFFCCF8091C6000895FC0190819923AF
:1012B00069F02DE09A3059F031968091C00085FF99
:1012C000FCCF9093C60090819923A1F70895809157
:1012D000C00085FFFCCF2093C600EECFFC019491A7
:1012E000992369F02DE09A3059F08091C00085FF74
:1012F000FCCF9093C600319694919923A1F708955D
:101300008091C00085FFFCCF2093C600EECF8134D2
:1013100014F087530895805308950F931F93DF931C
:10132000CF9300D00F92CDB7DEB790E09F938F930D
:1013300088E091E09F938F938E010F5F1F4F1F9363
:101340000F930E94DD3899812DB73EB72A5F3F4F3A
:101350000FB6F8943EBF0FBE2DBF992371F0F80170
:101360002DE09A3091F031968091C00085FFFCCF3E
:101370009093C60090819923A1F70F900F900F9042
:10138000CF91DF911F910F9108958091C00085FF4B
:10139000FCCF2093C600E7CF892B69F42B9885E01A
:1013A000982F9A95F1F72C9A982F9A95F1F72C98F7
:1013B0008A95F1F708952B9AF2CF181619065CF565
:1013C000672BA9F440E050E035E02B98232F2A95B5
:1013D000F1F72C9A232F2A95F1F72C98232F2A9591
:1013E000F1F74F5F5F4F4817590779F7089540E0CD
:1013F00050E035E02B9A232F2A95F1F72C9A232FD2
:101400002A95F1F72C98232F2A95F1F74F5F5F4F1C
:101410004817590779F70895AF92BF92CF92DF929C
:10142000EF92FF920F931F93E0EDF7E03197F1F702
:101430002A98AA2797FDA095BA2FBC01CD010E943A
:101440002F365B016C0120E030E04AEF54E40E944B
:10145000A5347B018C0120E030E040E85FE30E948E
:10146000FF358823A4F120E03FEF4FE757E4C801A0
:10147000B7010E949F351816ACF420E030E040E23E
:1014800051E4C601B5010E94A5340E94CF32CB01C0
:10149000672B79F028EC30E0F9013197F1F70197EB
:1014A000D9F707C0C801B7010E94CF32CB0101971D
:1014B000F1F72A9A80ED97E00197F1F71F910F91CC
:1014C000FF90EF90DF90CF90BF90AF90089561E0D4
:1014D00070E0ECCF18161906DCF440E050E035E07F
:1014E00013C02B9A232F2A95F1F72C9A232F2A9594
:1014F000F1F72C98232F2A95F1F74F5F5F4F48178C
:10150000590731F07595679560FDEBCF2B98EACFC1
:10151000089580B195E0292F2A95F1F72C9A292F6B
:101520002A95F1F72C989A95F1F7817008956F92AA
:101530007F928F929F92AF92BF92CF92DF92EF9263
:10154000FF920F931F93CF93DF9383E593E00E9465
:101550006E090E944E098230E1F7EE24FF2400E07C
:101560008824AA24BB249924CC24DD24E1E06E2E17
:10157000712C0E944E09182F882329F1133019F17C
:101580001A3209F49AC0083009F416C109300CF077
:1015900070C0043009F4F1C005300CF094C0023082
:1015A00009F4F5C0033029F7C12FD0E0CE01C09770
:1015B0008A30910508F0DEC07C0104E00E944E09EB
:1015C000182F8823D9F60E944E090E9487090E948D
:1015D0004E090E9487090E944E090E9487090E94B5
:1015E0004E090E94870994E0C91697E1D90609F0CF
:1015F0006DC128E1921609F0AAC1A114B10409F441
:10160000E8C1EE24FF248701A1E0B0E060E070E0D3
:1016100040E050E076956795FA01F595E795F595E8
:10162000E795F595E795E85DFC4F808190E0242FE4
:10163000277002C0959587952A95E2F780FF02C032
:1016400060587F4F4F5F5F4F37E14430530709F4D5
:10165000CFC11196A930B105E9F6CB01A0E0B0E009
:10166000E80EF91E0A1F1B1FA1E0B0E060E070E069
:10167000D1CF0C3009F477C00D30D4F50A3009F41D
:10168000BDC00B300CF4A9C0C12FD0E0CE01C09773
:101690000A9708F031C1C601880F991F880F991F5A
:1016A000880F991FCC0CDD1CC80ED91E80ED9FEF52
:1016B000C80ED91ECC0EDD1E5CCF81E593E00E94E2
:1016C0006E0902E056CF063009F4BDC007300CF4B5
:1016D000A3C0812F90E00E94DD3B892B09F049CF08
:1016E000103509F45DC1163409F46DC102E041CF33
:1016F0000E3041F10E30C4F00F3009F03ACF212FF7
:1017000030E0C901C0970A9708F008C1A294B294CA
:10171000B0EFBB22BA24AB22BA2480ED9FEFA80E13
:10172000B91EA20EB31E25CF812F90E00E94DD3B93
:10173000892B09F01ECF812F80538230D8F4882E58
:1017400001E017CFC12FD0E0CE010E94DD3B892BF5
:1017500009F00FCFCE01C0978A30910508F00FC174
:101760005C010FE006CF812F90E00E94DD3B892BCA
:1017700009F0FFCE20E030E0AFC0C12FD0E0CE01B5
:101780000E94DD3B892B09F48AC006E0F2CE812F4E
:1017900090E00E94DD3B892B09F0EBCE173409F471
:1017A00010C1183408F0DAC0133409F41DC116341E
:1017B00009F41CC101E0DDCE812F90E00E94DD3BE9
:1017C000892B09F0D6CE812F90E0C0970A9790F62A
:1017D00040ED942E910E0AE0CCCEC12FD0E0CE0188
:1017E0000E94DD3B892B09F0C4CECE01C0978A3020
:1017F000910508F0BFCF6C010BE0BBCE812F90E0CC
:10180000C0970A9708F081C01053392D3002C001EB
:101810001124912E980EADCEC12FD0E0CE010E94A2
:10182000DD3B892B09F0A5CE1053123008F0A2CF72
:10183000CE01C09741EE52E0BC0188E293E00E94E5
:10184000D63801E096CE812F90E00E94DD3B892BB7
:1018500009F08FCE812F8053823008F08BCFF701B3
:10186000F7FCB5C0F595E795F595E795F595E795FE
:10187000C70168E070E00E947F3B103309F493C019
:10188000E85DFC4F930102C0220F331F8A95E2F7F7
:101890008081822B80830894E11CF11C6ACECE01EA
:1018A000C0970A9708F066CFC701880F991F880F65
:1018B000991F880F991FEE0CFF1CE80EF91E20EDF2
:1018C0003FEFE20EF31EEC0EFD1E53CE88EF92E0CA
:1018D0000E946E0920E030E0C901DF91CF911F9195
:1018E0000F91FF90EF90DF90CF90BF90AF909F90BF
:1018F0008F907F906F900895812F90E00E94DD3B44
:10190000892B09F437CF0CE034CE812F90E00E9470
:10191000DD3B892B09F42ECF0CE02BCE812F90E0FC
:101920000E94E53B9C01815490400697F8F4C50164
:1019300082959295907F9827807F9827F9ECAF2E1B
:10194000FFEFBF2EA20EB31EA80EB91E12CE81EA63
:1019500092E00E946E0920E030E0BECF1C3409F412
:101960003FC0113509F026CF07E003CE812F90E06C
:101970000E94DD3B892B09F4FDCE02E0FACDCE01B9
:101980000E94E53B9C0181549040069708F0F2CEFE
:1019900019ECA12E1FEFB12EA20EB31E0FE0E9CD60
:1019A00008E09924E6CDE85DFC4F930102C0220FC8
:1019B000331F8A95E2F7C9018095208182238083B5
:1019C0006ACF0DE0D6CD09E0CC24DD24D2CD379608
:1019D00049CF8FE592E00E946E0920E030E07CCF95
:1019E000EE24FF2403E0C5CD0EE0C3CD05E0C1CD5C
:1019F00088E090E08A1B9B0B02C0769567958A95DC
:101A0000E2F76E0D7F1DA616B70631F481E0881649
:101A100051F021E030E060CF8FE492E00E946E0947
:101A200020E030E059CF82E192E00E946E0984ED1F
:101A300091E00E946E0981EA91E00E946E0983E6BE
:101A400091E00E946E09E5CFCF92DF92EF92FF9274
:101A50000F931F93DF93CF93CDB7DEB728970FB6C1
:101A6000F894DEBF0FBECDBF00E010E080E090E054
:101A7000FDE0CF2EF1E0DF2E7E010894E11CF11C89
:101A800020C0F801E85DFC4F808190E09F938F9328
:101A9000DF92CF92FF92EF920E94DD38C7010E9441
:101AA00055090F5F1F4FC8012DB73EB72A5F3F4F43
:101AB0000FB6F8943EBF0FBE2DBF32E0013E1307B4
:101AC00049F08F719070892BE1F686E593E00E94D2
:101AD0006E09D7CF28960FB6F894DEBF0FBECDBFE4
:101AE000CF91DF911F910F91FF90EF90DF90CF90FA
:101AF00008950F931F93DF93CF93CDB7DEB7C456EE
:101B0000D0400FB6F894DEBF0FBECDBFAC018091C0
:101B10000C0E90E08F7090708530910509F4B3C081
:101B200020910E0E8130910509F4BBC082309105E1
:101B30000CF4CAC08230910509F4C1C0039709F4BE
:101B4000B7C024E630E0309323032093220388ECCF
:101B500090E09093250380932403452B61F4CC59A6
:101B6000DF4F0FB6F894DEBF0FBECDBFCF91DF9130
:101B70001F910F91089560912603709127033F9361
:101B80002F93462F417089E14802A0011124CB0117
:101B9000969587958170907022E330E0FC01E29F7A
:101BA000C001E39F900DF29F900D1124480F842FE8
:101BB000992787FD90959F938F9377FD8FC075959B
:101BC0006795759567957F936F9381E191E09F93FA
:101BD0008F938E010F5F1F4F1F930F930E94DD386D
:101BE000C8010E9455098091160E90E09F938F9333
:101BF0008091150E90E09F938F938091140E90E04A
:101C00009F938F938091130E90E09F938F93809179
:101C1000120E90E09F938F938091110E90E09F930E
:101C20008F938091100E90E09F938F9380910F0E71
:101C300090E09F938F9380910E0E90E09F938F93EF
:101C400080910D0E90E09F938F9380910C0E90E009
:101C50009F938F9380910B0E90E09F938F938AE3D5
:101C600091E09F938F931F930F930E94DD388DB760
:101C70009EB786960FB6F8949EBF0FBE8DBFC80163
:101C80000E9455096CCF8091100E869590E08F715F
:101C900090700A96880F991F9093270380932603CC
:101CA00050CF8FE390E0909327038093260349CF92
:101CB00088E390E0909327038093260342CF2F3848
:101CC00081F08AE390E0F6CF892B09F03ACF82E4E5
:101CD00090E0909327038093260333CF6D5F7F4F6F
:101CE0006ECF8CE390E0E6CFBC015B9840984198C2
:101CF0002D982E982D9820E030E045E02B98842FE9
:101D00008A95F1F72C9A842F8A95F1F72C98842FD5
:101D10008A95F1F72F5F3F4F2438310579F760FF3F
:101D200068C02B9A85E0282F2A95F1F72C9A282F46
:101D30002A95F1F72C988A95F1F7AB0155954795BF
:101D400040FF61C02B9A85E0282F2A95F1F72C9A45
:101D5000282F2A95F1F72C988A95F1F755954795F4
:101D600040FF4FC02B9A85E0282F2A95F1F72C9A37
:101D7000282F2A95F1F72C988A95F1F755954795D4
:101D800040FF3DC02B9A85E0282F2A95F1F72C9A29
:101D9000282F2A95F1F72C988A95F1F755954795B4
:101DA00040FF2BC02B9A85E0282F2A95F1F72C9A1B
:101DB000282F2A95F1F72C988A95F1F741FF1BC03F
:101DC0002B9A85E0982F9A95F1F72C9A982F9A954F
:101DD000F1F72C988A95F1F780ED97E0FC013197A7
:101DE000F1F72A98FC013197F1F72A9A0197F1F758
:101DF00008952B9897CF2B98E4CF2B98D4CF2B987E
:101E0000C2CF2B98B0CF2B989ECF11B882E084B967
:101E100017B880E48AB99FEF92B98DEF85B998B968
:101E20008BB18F6B8BB985E38A95F1F75E9A20E0D1
:101E300030E048EC50E0CA010197F1F72F5F3F4FC7
:101E400083E0283E3807B9F720E23EE4C901019754
:101E5000F1F712B884E085B918B88BB180748BB9EA
:101E60008EEF81B98FEF84B983E087B98CED8AB9A1
:101E700080E49CE90197F1F72898C9010197F1F7EF
:101E80008AE390E00E94740EEBE0FEE025E0108211
:101E900080B1922F9A95F1F72C9A922F9A95F1F79B
:101EA0002C98922F9A95F1F780FF03C08081816072
:101EB000808380B1922F9A95F1F72C9A922F9A9560
:101EC000F1F72C98922F9A95F1F780FF03C080814B
:101ED0008260808380B1922F9A95F1F72C9A922F8D
:101EE0009A95F1F72C98922F9A95F1F780FF03C0FD
:101EF00080818460808380B1922F9A95F1F72C9A2B
:101F0000922F9A95F1F72C98922F9A95F1F780FFDE
:101F100003C080818860808380B1922F9A95F1F709
:101F20002C9A922F9A95F1F72C98922F9A95F1F777
:101F300080FF03C080818061808380B1922F9A9559
:101F4000F1F72C9A922F9A95F1F72C98922F9A9557
:101F5000F1F780FF03C080818062808380B1922F7F
:101F60009A95F1F72C9A922F9A95F1F72C98922F37
:101F70009A95F1F780FF03C080818064808380B1EF
:101F8000922F9A95F1F72C9A922F9A95F1F72C9817
:101F9000922F9A95F1F780FF03C08081806880833B
:101FA00031968EE0E531F80709F071CF80E991E0D4
:101FB0000197F1F711B882E084B917B880E48AB9C3
:101FC0009FEF92B98DEF85B998B98BB18F6B8BB9B3
:101FD00080E29EE40197F1F75E9885E38A95F1F738
:101FE00008952F923F924F925F926F927F928F92BD
:101FF0009F92AF92BF92CF92DF92EF92FF920F9398
:102000001F93DF93CF93CDB7DEB728970FB6F89421
:10201000DEBF0FBECDBF888711B882E084B917B884
:1020200080E48AB99FEF92B98DEF85B998B98BB1E9
:102030008F6B8BB985E38A95F1F75E9A20E030E0EB
:1020400048EC50E0CA010197F1F72F5F3F4F83E062
:10205000283E3807B9F720E23EE4C9010197F1F7BD
:1020600012B884E085B918B88BB180748BB98EEF43
:1020700081B98FEF84B983E087B98CED8AB980E4A8
:102080009CE90197F1F72898C9010197F1F7809130
:10209000A6019091A701181619060CF0BDC3AA2439
:1020A000BB2422243324CC2495E0D92E80ED482E65
:1020B00087E0582E01E0602E712C5B984098419883
:1020C0002D982E982D9820E030E02B988D2D8A9514
:1020D000F1F72C9A8D2D8A95F1F72C988D2D8A95F4
:1020E000F1F72F5F3F4F2438310579F7A0FE46C145
:1020F0002B9A8D2D8A95F1F72C9A8D2D8A95F1F7D3
:102100002C988D2D8A95F1F795013595279520FF0F
:102110003DC12B9A8D2D8A95F1F72C9A8D2D8A959C
:10212000F1F72C988D2D8A95F1F73595279520FF9D
:102130002BC12B9A8D2D8A95F1F72C9A8D2D8A958E
:10214000F1F72C988D2D8A95F1F73595279520FF7D
:1021500019C12B9A8D2D8A95F1F72C9A8D2D8A9580
:10216000F1F72C988D2D8A95F1F73595279520FF5D
:1021700007C12B9A8D2D8A95F1F72C9A8D2D8A9572
:10218000F1F72C988D2D8A95F1F721FFF5C02B9A48
:102190008D2D8A95F1F72C9A8D2D8A95F1F72C9833
:1021A0008D2D8A95F1F7C2010197F1F72A98C201A6
:1021B0000197F1F72A9AC2010197F1F78090A801DF
:1021C0009090A901181419040CF040C0E090A601E9
:1021D000F090A7019885992309F0DAC000E010E09B
:1021E000E09EC001E19E900DF09E900D11248A0D9D
:1021F0009B1D9C0197FDBDC035952795359527956D
:102200003595279568E070E00E947F3B482F80B1AC
:102210009D2D9A95F1F72C9A9D2D9A95F1F72C9872
:102220009D2D9A95F1F780FF96C0C30102C0880FDB
:10223000991F4A95E2F7F901E85DFC4F9081982BD0
:1022400090830F5F1F4F0815190554F20894A11CC5
:10225000B11C8091A6019091A701A816B9060CF4B3
:102260002CCF8091AA019091AB010E94740E8091B5
:10227000AE019091AF01181619060CF04FC12885D8
:10228000222309F40AC100E010E0A5E0DA2EF1E013
:10229000AF2EB12CE4E66E2EE1E07E2E4E010894C6
:1022A000811C911C2BC0C501042E02C0880F991FF0
:1022B0000A94E2F7C82A8C2D992787FD9095F7019B
:1022C000E85DFC4F208130E082279327042E02C076
:1022D000959587950A94E2F780FD7EC20F5F1F4FA8
:1022E0008091AE019091AF01880F991F880F991FBF
:1022F000880F991F081719070CF010C18091AC01C5
:102300009091AD01800F911FFC0197FD42C27F01AA
:10231000F594E794F594E794F594E79468E070E019
:102320000E947F3BAC0180B19D2D9A95F1F72C9ACC
:102330009D2D9A95F1F72C989D2D9A95F1F780FD9A
:10234000B2CFC501042E02C0880F991F0A94E2F78C
:102350008095C822B0CFC30102C0880F991F4A954B
:10236000E2F7982F9095F901E85DFC4F8081982362
:1023700067CF295F3F4F40CF2B980ACF2B98B9CE1C
:102380002B98F8CE2B98E6CE2B98D4CE2B98C2CE95
:1023900000E010E029C0C301042E02C0880F991F7D
:1023A0000A94E2F7C82A8C2D992787FD9095F701AA
:1023B000E85DFC4F208130E082279327042E02C085
:1023C000959587950A94E2F780FD40C00F5F1F4FF7
:1023D0008091A8019091A901081719070CF036CF38
:1023E000E090A601F090A7010E9DC0010F9D900DF9
:1023F0001E9D900D11248A0D9B1DFC0197FD24C08C
:102400007F01F594E794F594E794F594E79468E0F8
:1024100070E00E947F3BAC0180B19D2D9A95F1F751
:102420002C9A9D2D9A95F1F72C989D2D9A95F1F760
:1024300080FDB1CFC301042E02C0880F991F0A94FA
:10244000E2F78095C822AFCF3796DACFC701880F61
:10245000991F880F991F880F991F840F951F9F93AD
:102460008F9384E691E09F938F9381E090E08C0FAF
:102470009D1F9F938F930E94DD38CE0101960E948D
:10248000550931E0232E312C8DB79EB706960FB635
:10249000F8949EBF0FBE8DBF99CF00E010E05C01A5
:1024A000AA0CBB1CAA0CBB1CAA0CBB1C95E0F92EE9
:1024B00081E0882E912C8091AC019091AD01800F2C
:1024C000911F9C0197FD62C13595279535952795FC
:1024D0003595279568E070E00E947F3B482F80B1DA
:1024E0009F2D9A95F1F72C9A9F2D9A95F1F72C989C
:1024F0009F2D9A95F1F780FF39C1C40102C0880F62
:10250000991F4A95E2F7F901E85DFC4F9081982BFD
:1025100090830F5F1F4F0A151B056CF28091B80165
:1025200080FF14C15B9A81FF0FC1409A82FF0AC1EC
:10253000419A83FF05C12F9A84FFFDC02E9A85FD25
:10254000FDC02D9880ED97E0FC013197F1F72A98B6
:10255000E0EAFFE03197F1F72A9A0197F1F7A090AE
:10256000BC01B090BD011A141B040CF0B0C09885DA
:10257000992309F46AC0EE24FF24B5E0DB2EA1E024
:10258000AA2EB12CF4E66F2EF1E07F2E4E010894B6
:10259000811C911C26C0C501042E02C0880F991F02
:1025A0000A94E2F7C82A8C2D992787FD9095F801A7
:1025B000E85DFC4F208130E082279327042E02C083
:1025C000959587950A94E2F780FDE7C00894E11C91
:1025D000F11C8091BC019091BD01E816F9060CF048
:1025E00076C0C701880F991FE091BA01F091BB0135
:1025F000E80FF91F408151819A01C90137FDCBC015
:102600008C01159507951595079515950795CA01A0
:1026100068E070E00E947F3BAC0180B19D2D9A95EF
:10262000F1F72C9A9D2D9A95F1F72C989D2D9A955E
:10263000F1F780FDB0CFC501042E02C0880F991FAD
:102640000A94E2F78095C822AECF00E010E0C09077
:10265000BA01D090BB0135E0F32E21E0822E912CFF
:10266000F801EE0FFF1FEC0DFD1D408151819A0115
:10267000C90137FD89C09C0135952795359527956A
:1026800035952795CA0168E070E00E947F3B482F8E
:1026900080B19F2D9A95F1F72C9A9F2D9A95F1F77D
:1026A0002C989F2D9A95F1F780FF52C0C40102C06B
:1026B000880F991F4A95E2F7F901E85DFC4F908178
:1026C000982B90830F5F1F4F0A151B054CF280E972
:1026D00091E00197F1F711B882E084B917B880E46E
:1026E0008AB99FEF92B98DEF85B998B98BB18F6B8D
:1026F0008BB980E29EE40197F1F75E9885E38A95B5
:10270000F1F7C10128960FB6F894DEBF0FBECDBF1A
:10271000CF91DF911F910F91FF90EF90DF90CF90BD
:10272000BF90AF909F908F907F906F905F904F90F1
:102730003F902F9008952E9885FF03CF2D9A02CFBA
:102740002D98FACE4198F5CE4098F0CE5B98EBCE1E
:10275000C40102C0880F991F4A95E2F7982F9095FF
:10276000F901E85DFC4F80819823ABCFC40102C022
:10277000880F991F4A95E2F7982F9095F901E85D27
:10278000FC4F80819823C4CE079675CF295F3F4FB9
:102790009BCE3796BCCD079633CF000F111F000F8D
:1027A000111F000F111F040F151F1F930F937F920E
:1027B0006F929F928F920E94DD38C4010E9455094A
:1027C00041E0242E312C8DB79EB706960FB6F894B3
:1027D0009EBF0FBE8DBFFACEC701880F991F880F0D
:1027E000991F880F991F840F951F9F938F937F9236
:1027F0006F929F928F920E94DD38C4010E9455090A
:1028000051E0252E312C8DB79EB706960FB6F89461
:102810009EBF0FBE8DBF62CD22243324CC2421CD98
:10282000AF92BF92CF92DF92EF92FF920F931F93DE
:1028300011B882E084B917B880E48AB99FEF92B9E1
:102840008DEF85B998B98BB18F6B8BB985E38A957C
:10285000F1F75E9A20E030E048EC50E0CA010197C1
:10286000F1F72F5F3F4F83E0283E3807B9F720E2AA
:102870003EE4C9010197F1F712B884E085B918B8B0
:102880008BB180748BB98EEF81B98FEF84B983E0FF
:1028900087B98CED8AB980E49CE90197F1F7289A11
:1028A000C9010197F1F75B9A4098419A2F9A2E9AA5
:1028B0002D9A80ED97E00197F1F72A986091240313
:1028C00070912503882777FD8095982F0E942F36D9
:1028D0005B016C0120E030E04AEF54E40E94A53433
:1028E0007B018C0120E030E040E85FE30E94FF358F
:1028F000882304F120E03FEF4FE757E4C801B70118
:102900000E949F3518160CF042C020E030E040E2F3
:1029100051E4C601B5010E94A5340E94CF32CB011B
:10292000672B69F028EC30E0F9013197F1F7019756
:10293000D9F705C061E070E0CB010197F1F72A9A61
:1029400080ED97E00197F1F780E991E00197F1F7C9
:1029500011B882E084B917B880E48AB99FEF92B9C0
:102960008DEF85B998B98BB18F6B8BB980E29EE4FE
:102970000197F1F75E9885E38A95F1F71F910F9122
:10298000FF90EF90DF90CF90BF90AF900895C80177
:10299000B7010E94CF32D0CF2F923F924F925F92D9
:1029A0006F927F929F92AF92BF92CF92DF92EF92FF
:1029B000FF920F931F93DF93CF93CDB7DEB7289786
:1029C0000FB6F894DEBF0FBECDBF9A83898311B8CE
:1029D00082E084B917B880E48AB99FEF92B98DEF8D
:1029E00085B998B98BB18F6B8BB985E38A95F1F76F
:1029F0005E9A20E030E048EC50E0CA010197F1F720
:102A00002F5F3F4F83E0283E3807B9F720E23EE4CE
:102A1000C9010197F1F712B884E085B918B88BB1F4
:102A200080748BB98EEF81B98FEF84B983E087B959
:102A30008CED8AB980E49CE90197F1F7289AC901E5
:102A40000197F1F75B98409841982D982E982D9812
:102A50002090A6013090A701121413040CF059C362
:102A60006090A8017090A901A0912203B091230366
:102A7000B887AF8344245524CD01AA2797FDA0959C
:102A8000BA2F8B839C83AD83BE8375E0972E16147B
:102A90001704ACF5A981BA81AB2B09F09BC2720176
:102AA00000E010E0A701F701F7FC86C2F595E79575
:102AB000F595E795F595E795E85DFC4F208130E0C9
:102AC000CA0168E070E00E947F3B02C035952795FF
:102AD0008A95E2F720FF6EC22B9A892D8A95F1F72D
:102AE0002C9A892D8A95F1F72C98892D8A95F1F7E2
:102AF0000F5F1F4FE20CF31C061517059CF240FCFC
:102B00005FC22B98892D8A95F1F72C9A892D8A9589
:102B1000F1F72C98892D8A95F1F792013595279533
:102B200020FD56C22B98892D8A95F1F72C9A892D74
:102B30008A95F1F72C98892D8A95F1F73595279587
:102B400020FD44C22B98892D8A95F1F72C9A892D66
:102B50008A95F1F72C98892D8A95F1F73595279567
:102B600020FD32C22B98892D8A95F1F72C9A892D58
:102B70008A95F1F72C98892D8A95F1F73595279547
:102B800020FD20C22B98892D8A95F1F72C9A892D4A
:102B90008A95F1F72C98892D8A95F1F721FF0EC2BD
:102BA0002B9A892D8A95F1F72C9A892D8A95F1F720
:102BB0002C98892D8A95F1F72B9880ED97E0019755
:102BC000F1F72A986B817C818D819E810E942F363E
:102BD0005B016C0120E030E04AEF54E40E94A53430
:102BE0007B018C0120E030E040E85FE30E94FF358C
:102BF00088230CF40BC220E03FEF4FE757E4C801F5
:102C0000B7010E949F3518160CF0F8C120E030E0A3
:102C100040E251E4C601B5010E94A5340E94CF32C2
:102C2000CB01672B31F0E8ECF0E03197F1F7019739
:102C3000D1F72A9A80ED97E00197F1F70894411CAB
:102C4000511C421453040CF422CF0091AE01109198
:102C5000AF01000F111F000F111F000F111F1016E1
:102C600011060CF039C0E090AC01F090AD01298163
:102C70003A81232B09F0CFC1CC24DD2445E0C601E5
:102C80008E0D9F1DFC0197FDFEC1F595E795F5950D
:102C9000E795F595E795E85DFC4F208130E068E029
:102CA00070E00E947F3B02C0359527958A95E2F738
:102CB00020FFE7C12B9A842F8A95F1F72C9A842F55
:102CC0008A95F1F72C98842F8A95F1F70894C11C06
:102CD000D11CC016D1069CF2061517050CF4B3C121
:102CE0002091AA013091AB0120FD93C12B9885E082
:102CF000982F9A95F1F72C9A982F9A95F1F72C988E
:102D00008A95F1F73595279520FDC9C12B9885E067
:102D1000982F9A95F1F72C9A982F9A95F1F72C986D
:102D20008A95F1F73595279520FDB7C12B9885E059
:102D3000982F9A95F1F72C9A982F9A95F1F72C984D
:102D40008A95F1F73595279520FDA5C12B9885E04B
:102D5000982F9A95F1F72C9A982F9A95F1F72C982D
:102D60008A95F1F73595279520FD93C12B9885E03D
:102D7000982F9A95F1F72C9A982F9A95F1F72C980D
:102D80008A95F1F721FF83C12B9A85E0982F9A95B8
:102D9000F1F72C9A982F9A95F1F72C988A95F1F7DC
:102DA0002B9880ED97E00197F1F72A98AF81B885CD
:102DB000BD01882777FD8095982F0E942F362B0123
:102DC0003C0120E030E04AEF54E40E94A5345B016E
:102DD0006C0120E030E040E85FE30E94FF3588238B
:102DE0000CF491C120E03FEF4FE757E4C601B50175
:102DF0000E949F3518160CF076C120E030E040E2CA
:102E000051E4C301B2010E94A5340E94CF32CB012C
:102E1000672B39F028EC30E0F9013197F1F7019791
:102E2000D9F72A9A80ED97E00197F1F78091B801E0
:102E300080FF42C15B9A81FF3DC1409A82FF38C149
:102E4000419A83FF33C12F9A84FF2BC12E9A85FDAF
:102E50002BC12D98E090BC01F090BD011E141F0401
:102E60000CF041C02091BA013091BB01E981FA8197
:102E7000EF2B09F023C1190100E010E035E0932E9B
:102E8000D1014C9111965C91CA01FC0197FDFDC0E6
:102E9000F595E795F595E795F595E795E85DFC4F90
:102EA000208130E0CA0168E070E00E947F3B02C0F0
:102EB000359527958A95E2F720FFE1C02B9A892D59
:102EC0008A95F1F72C9A892D8A95F1F72C98892DFE
:102ED0008A95F1F70F5F1F4FE2E0F0E02E0E3F1EE4
:102EE0000E151F056CF22B9880ED97E00197F1F716
:102EF0002A9820E030E040E85FE3C601B5010E9477
:102F0000FF3588230CF402C120E03FEF4FE757E480
:102F1000C601B5010E949F3518160CF0ECC020E0E8
:102F200030E040E251E4C301B2010E94A5340E94A6
:102F3000CF32CB01672B39F028EC30E0F901319723
:102F4000F1F70197D9F72A9A80ED97E00197F1F709
:102F500080E991E00197F1F711B882E084B917B8E0
:102F600080E48AB99FEF92B98DEF85B998B98BB19A
:102F70008F6B8BB980E29EE40197F1F75E9885E351
:102F80008A95F1F728960FB6F894DEBF0FBECDBF35
:102F9000CF91DF911F910F91FF90EF90DF90CF9035
:102FA000BF90AF909F907F906F905F904F903F90B9
:102FB0002F9008952B9891CD379678CD2B98F1CD01
:102FC0002B9AA0CD2B9ADFCD2B9ACDCD2B9ABBCDB2
:102FD0002B9AA9CD20E030E02B9A892D8A95F1F724
:102FE0002C9A892D8A95F1F72C98892D8A95F1F7DD
:102FF0002F5F3F4F261537057CF381CDC801B70100
:103000000E94CF32CB010197F1F713CE61E070E05F
:10301000F9CF2B9A6CCE20E030E095E02B9A892FE7
:103020008A95F1F72C9A892F8A95F1F72C98892F98
:103030008A95F1F72F5F3F4F201731077CF3061574
:1030400017050CF04DCEA301401B510B14161506AD
:103050000CF046CE20E030E095E02B98892F8A9541
:10306000F1F72C9A892F8A95F1F72C98892F8A9558
:10307000F1F72F5F3F4F2417350779F731CE2B98A3
:103080001ECF2B9818CE379600CE379601CF2B98AF
:103090007CCE2B9A6CCE2B9A5ACE2B9A48CE2B9A5A
:1030A00036CE2E9885FFD5CE2D9AD4CE2D98CCCE67
:1030B0004198C7CE4098C2CE5B98BDCE20E030E0AC
:1030C00095E02B9A892F8A95F1F72C9A892F8A956A
:1030D000F1F72C98892F8A95F1F72F5F3F4F2E1526
:1030E0003F057CF300CFC601B5010E94CF32CB0172
:1030F0000197F1F796CEC601B5010E94CF32CB0100
:103100000197F1F720CF61E070E0F1CF61E070E06E
:10311000F6CF6090A8017090A901E0912203F09190
:103120002303F887EF8391CD85B78F7E85BF11B8D4
:1031300082E084B917B880E48AB98DEF85B98FEF42
:1031400082B988B98FEB8BB90895329B0BC01E9B57
:1031500005C086B120E030E0C901089521E030E0EB
:10316000C901089522E030E0C90108952F923F92ED
:103170004F925F926F927F928F929F92AF92BF9287
:10318000CF92DF92EF92FF920F931F93DF93CF9333
:10319000CDB7DEB764970FB6F894DEBF0FBECDBFD4
:1031A00084E999E00E946E090E944E098A33E1F792
:1031B0000E944E090E948709582E529460EF5622B1
:1031C0000E944E090E948709582A0E944E090E94B7
:1031D0008709F82EF29450EFF5220E944E090E94C2
:1031E0008709F82A0E944E090E948709182F129514
:1031F000107F0E944E090E948709182B0E944E09D9
:103200000E948709482E429440EF44220E944E09B2
:103210000E948709482A0F2D050D010F040D81E03A
:10322000841508F46EC0552009F48CC0812F90E0FD
:103230003F2C22243101680E791E730137E9C32E19
:103240003EE0D32EC80ED91E27E1822E2EE0922E0C
:10325000880E991E8BE0A82E86E0B82EA60CB71C0F
:1032600014C0F6011083010F0894E11CF11C0894AE
:10327000C11CD11C0894811C911C0894A11CB11C78
:103280008E2D8619851508F05DC00E944E090E949A
:103290008709182F1295107F0E944E090E948709F6
:1032A000182BC701805090444097D8F2C701805036
:1032B00092448138910518F4F4011083D4CFF0E0E2
:1032C000EF16F8E0FF060CF05BC080910906813034
:1032D00019F0F5011083C7CF80910A068D3311F0E4
:1032E0008238B9F781E0E81684E0F80690F389EABD
:1032F00098E00E946E098AE798E00E946E098FEFBD
:1033000048C085E799E00E946E09842D90E09F9364
:103310008F93E6E0F2E0FF93EF9381E090E08C0F73
:103320009D1F9F938F930E94DD38CE0101960E94CE
:103330005509EDB7FEB736960FB6F894FEBF0FBE2F
:10334000EDBF32CF0E944E090E948709182F1295B7
:10335000107F0E944E090E948709182B01950117C2
:1033600051F4F1E04F1611F4552061F182E598E037
:103370000E946E0919CF84E598E00E946E09F1CF92
:103380008DE299E00E946E098AEE98E00E946E0933
:103390008FEF64960FB6F894DEBF0FBECDBFCF910E
:1033A000DF911F910F91FF90EF90DF90CF90BF9032
:1033B000AF909F908F907F906F905F904F903F90D5
:1033C0002F9008950E944E0980E0E3CF0F931F9342
:1033D00085B78F7E85BF11B812E014B917B880E4A5
:1033E0008AB98DEF85B90FEF02B908B98FEB8BB9A8
:1033F0001092C50083E38093C40088E18093C100EC
:1034000086E08093C2008091C200877F8093C200D3
:103410000E944E098AE298E00E946E09329BB8C170
:103420001E9B9CC186B11092090686E997E00E9416
:103430006E0901B904B917B815B812B80E94A606EA
:1034400080910906882309F067C1EBE0F6E011924C
:103450002EE0EB30F207D9F786E797E00E946E097D
:103460000E944E09992787FD90950E94E53B182FF1
:103470000E94460980910906813099F0823009F155
:10348000133409F4A7C014347CF51D3029F311342A
:1034900009F49BC01A3001F388E593E00E946E099D
:1034A000DBCF143449F1153454F51D30A9F21E3028
:1034B0000CF0B0C01A3081F28FE596E00E946E09E0
:1034C000CBCF143409F410C115340CF041C01D30B9
:1034D00019F21E300CF0DEC01A3009F4BDCF88E6B8
:1034E00094E00E946E09B8CF183409F476C01934FC
:1034F0000CF063C0143481F60E94B618ADCF1035BD
:1035000009F44EC011350CF08DC01834A9F689E6C7
:1035100097E00E946E0984E597E00E946E0981E4BD
:1035200097E00E946E0985E197E00E946E0980EFA6
:1035300096E00E946E0980ED96E00E946E098DE98A
:1035400096E00E946E0980E796E00E946E0984CFA3
:10355000103509F478C011350CF0B0C0183409F0FA
:10356000BECF83E395E00E946E098EE195E00E9454
:103570006E098BE095E00E946E0984EE94E00E9453
:103580006E098DEB94E00E946E0989E994E00E9437
:103590006E0989E794E00E946E095ECF0E94B6181A
:1035A0000E94F9300E943D1E97FD56CF0E942420B4
:1035B00097FD52CF0E94712A4FCF103541F016353A
:1035C00009F06ACF0E94960747CF0E94B6180E9462
:1035D0005F0842CF0E940E073FCF8BE594E00E9428
:1035E0006E0989E394E00E946E0989E194E00E94EB
:1035F0006E098DEE93E00E946E0982EC93E00E94CA
:103600006E0982EA93E00E946E0989E693E00E94C7
:103610006E0922CF113411F2133409F04DCF0E94FC
:10362000F9301ACF153599F1163509F045CF0E94BA
:10363000D92112CF0E94970A892B09F468C085EF1F
:1036400095E00E946E0980E090E00E94790D85EA85
:1036500095E00E946E090E94101489E995E00E948D
:103660006E0985E895E00E946E0980E090E00E9476
:10367000CC1486E695E00E946E0981E00E94F10F6D
:10368000892BD9F182E595E00E946E09E5CE0E9472
:10369000C92CE2CE113471F2133409F020CF80E04E
:1036A00090E00E94790D8FE496E00E946E090E94DE
:1036B000101483E496E00E946E09CECE143569F0B2
:1036C000163509F00CCF80E090E00E94790D80E083
:1036D0000E94F10F0E94240DBFCE0E94050F81E0D1
:1036E00090E00E94790DB8CE0E94970A892B51F084
:1036F0008AE296E00E946E09AFCE80E495E00E94D7
:103700006E09AACE8EE096E00E946E09A5CE85EBEA
:1037100095E00E946E09A0CE813009F09DCEEBE0CD
:10372000F6E08FEF9FE38083918332962EE0EB30BB
:10373000F207C9F7E7E1FEE08FEF81939EE0E739FA
:10374000F907D9F7E7E9FEE08FEF9FE380839183E4
:1037500032962EE0E73AF207C9F77ECE81E08093F9
:10376000090688E198E00E946E0984E884B911B9DD
:103770000E94AE2780910A06882309F061CE81ED70
:1037800097E00E946E098FEA97E00E946E09FFCFD2
:10379000109309068FE797E00E946E0951CE4F9271
:1037A0005F926F927F928F929F92AF92BF92CF92D1
:1037B000DF92EF92FF920F931F93CF93DF930A98BC
:1037C000119A85E0982F9A95F1F71198982F9A956C
:1037D000F1F7119A982F9A95F1F720B1982F9A95B1
:1037E000F1F71198982F9A95F1F7119A8A95F1F7B8
:1037F0000299F9C04424552485E0982F9A95F1F751
:103800001198982F9A95F1F7119A982F9A95F1F7A8
:1038100090B1482F4A95F1F71198482F4A95F1F742
:10382000119A8A95F1F7029901C16624772485E0FF
:10383000482F4A95F1F71198482F4A95F1F7119AB8
:103840008A95F1F70299EEC08824992485E0482FE3
:103850004A95F1F71198482F4A95F1F7119A8A95F0
:10386000F1F70299DBC0AA24BB2485E0482F4A95D2
:10387000F1F71198482F4A95F1F7119A8A95F1F7C7
:103880000299C8C0CC24DD2485E0482F4A95F1F781
:103890001198482F4A95F1F7119A8A95F1F70299F4
:1038A000B5C0EE24FF2485E0482F4A95F1F7119822
:1038B000482F4A95F1F7119A8A95F1F70299A3C01A
:1038C00000E010E085E0482F4A95F1F71198482F65
:1038D0004A95F1F7119A8A95F1F7029991C0C0E0E3
:1038E000D0E085E0482F4A95F1F71198482F4A9586
:1038F000F1F7119A8A95F1F702997FC0A0E0B0E044
:1039000085E0482F4A95F1F71198482F4A95F1F72D
:10391000119A8A95F1F702996DC0E0E0F0E085E038
:10392000482F4A95F1F71198482F4A95F1F7119AC7
:103930008A95F1F702995BC060E070E085E0482F5E
:103940004A95F1F71198482F4A95F1F7119A8A95FF
:10395000F1F702996FC040E050E030E036952795CE
:103960003695279521703070892F90E08470907083
:10397000282B392B24293529262937292829392983
:103980002A293B292C293D292E293F29202B312B5F
:103990002C2B3D2B2A2B3B2B2E2B3F2B262B372B37
:1039A00085E0982F9A95F1F71198982F9A95F1F74D
:1039B000119A8A95F1F7119882E08A95F1F7242BF4
:1039C000352BC901DF91CF911F910F91FF90EF909F
:1039D000DF90CF90BF90AF909F908F907F906F902F
:1039E0005F904F900895E2E04E2E512C05CF60E09D
:1039F00070E1A4CFE0E0F8E092CFA0E0B4E080CFA7
:103A0000C0E0D2E06ECF00E011E05CCF30E8E32E02
:103A1000F12C49CF40E4C42ED12C36CF50E2A52E54
:103A2000B12C23CF60E1862E912C10CF78E0672E49
:103A3000712CFDCE40E050E290CFAC010A9A119A71
:103A4000129885E0282F2A95F1F71198282F2A95AA
:103A5000F1F7119A8A95F1F740FFE5C082B18460D1
:103A600082B985E0282F2A95F1F71198282F2A95F9
:103A7000F1F7119A8A95F1F741FFF9C082B184609C
:103A800082B985E0282F2A95F1F71198282F2A95D9
:103A9000F1F7119A8A95F1F742FFE6C082B184608E
:103AA00082B985E0282F2A95F1F71198282F2A95B9
:103AB000F1F7119A8A95F1F743FFD3C082B1846080
:103AC00082B985E0282F2A95F1F71198282F2A9599
:103AD000F1F7119A8A95F1F744FFC0C082B1846072
:103AE00082B985E0282F2A95F1F71198282F2A9579
:103AF000F1F7119A8A95F1F745FFADC082B1846064
:103B000082B985E0282F2A95F1F71198282F2A9558
:103B1000F1F7119A8A95F1F746FF9AC082B1846055
:103B200082B985E0282F2A95F1F71198282F2A9538
:103B3000F1F7119A8A95F1F747FF87C082B1846047
:103B400082B985E0282F2A95F1F71198282F2A9518
:103B5000F1F7119A8A95F1F750FF74C082B1846031
:103B600082B985E0282F2A95F1F71198282F2A95F8
:103B7000F1F7119A8A95F1F751FF61C082B1846023
:103B800082B985E0282F2A95F1F71198282F2A95D8
:103B9000F1F7119A8A95F1F752FF4EC082B1846015
:103BA00082B985E0282F2A95F1F71198282F2A95B8
:103BB000F1F7119A8A95F1F753FF3BC082B1846007
:103BC00082B985E0282F2A95F1F71198282F2A9598
:103BD000F1F7119A8A95F1F754FF28C082B18460F9
:103BE00082B985E0282F2A95F1F71198282F2A9578
:103BF000F1F7119A8A95F1F755FD3CC082B18B7FA0
:103C000082B985E0982F9A95F1F71198982F9A9597
:103C1000F1F7119A8A95F1F7129811980A9882E0B3
:103C20008A95F1F7089582B18B7F1ACF82B18B7F8D
:103C3000D7CF82B18B7FC4CF82B18B7FB1CF82B11E
:103C40008B7F9ECF82B18B7F8BCF82B18B7F78CFE2
:103C500082B18B7F65CF82B18B7F52CF82B18B7F58
:103C60003FCF82B18B7F2CCF82B18B7F19CF82B1B6
:103C70008B7F06CF82B18460C3CF6F927F928F9289
:103C80009F92AF92BF92CF92DF92EF92FF920F93EB
:103C90001F93CF93DF9311982A982F988DE0982F38
:103CA0009A95F1F72A9A982F9A95F1F72F9A8A9573
:103CB000F1F78FEA9CE00E946E09CBE0D6E0AA24DF
:103CC000BB2415E002E0A0E48A2EAFE19A2EF0E8D2
:103CD0006F2EFEE37F2E44C1F980EE249701207001
:103CE0003F73888190E0282B392B8FE32F3F3807D3
:103CF00009F4E8C00A9A119A1298812F8A95F1F76F
:103D00001198812F8A95F1F7119A812F8A95F1F7F1
:103D1000129A812F8A95F1F71198812F8A95F1F7E0
:103D2000119A812F8A95F1F71298812F8A95F1F7D0
:103D30001198812F8A95F1F7119A812F8A95F1F7C1
:103D40001298812F8A95F1F71198812F8A95F1F7B2
:103D5000119A812F8A95F1F71298812F8A95F1F7A0
:103D60001198812F8A95F1F7119A812F8A95F1F791
:103D7000129811980A98802F8A95F1F7C9010E942C
:103D80001D1D80910A068D53823008F4F4C00A9AF2
:103D9000119A1298812F8A95F1F71198812F8A959F
:103DA000F1F7119A812F8A95F1F71298812F8A9550
:103DB000F1F71198812F8A95F1F7119A812F8A9541
:103DC000F1F71298812F8A95F1F71198812F8A9532
:103DD000F1F7119A812F8A95F1F7129A812F8A951E
:103DE000F1F71198812F8A95F1F7119A812F8A9511
:103DF000F1F71298812F8A95F1F71198812F8A9502
:103E0000F1F7119A812F8A95F1F7129811980A9873
:103E1000802F8A95F1F7C4010197F1F70A9A119A58
:103E20001298812F8A95F1F71198812F8A95F1F7D1
:103E3000119A812F8A95F1F71298812F8A95F1F7BF
:103E40001198812F8A95F1F7119A812F8A95F1F7B0
:103E5000129A812F8A95F1F71198812F8A95F1F79F
:103E6000119A812F8A95F1F71298812F8A95F1F78F
:103E70001198812F8A95F1F7119A812F8A95F1F780
:103E80001298812F8A95F1F71198812F8A95F1F771
:103E9000119A812F8A95F1F7129811980A98802F1C
:103EA0008A95F1F70E94CF1BD980CC24960120700F
:103EB0003F73488150E0242B352B9F738217930763
:103EC00009F0A1C00A9A119A1298812F8A95F1F7E8
:103ED0001198812F8A95F1F7119A812F8A95F1F720
:103EE000129A812F8A95F1F71198812F8A95F1F70F
:103EF000119A812F8A95F1F7129A812F8A95F1F7FD
:103F00001198812F8A95F1F7119A812F8A95F1F7EF
:103F10001298812F8A95F1F71198812F8A95F1F7E0
:103F2000119A812F8A95F1F71298812F8A95F1F7CE
:103F30001198812F8A95F1F7119A812F8A95F1F7BF
:103F4000129811980A98802F8A95F1F70894A11C6D
:103F5000B11C229680E0A81684E0B80609F46FC070
:103F6000C5018F719070892B09F0B6CE8DEA9CE067
:103F70000E946E09B1CE0A9A119A1298812F8A95E1
:103F8000F1F71198812F8A95F1F7119A812F8A956F
:103F9000F1F71298812F8A95F1F71198812F8A9560
:103FA000F1F7119A812F8A95F1F71298812F8A954E
:103FB000F1F71198812F8A95F1F7119A812F8A953F
:103FC000F1F7129A812F8A95F1F71198812F8A952E
:103FD000F1F7119A812F8A95F1F7129A812F8A951C
:103FE000F1F71198812F8A95F1F7119A812F8A950F
:103FF000F1F7129811980A98802F8A95F1F7C3016A
:104000000197F1F70BCF85E89CE00E946E0984E6EA
:104010009CE00E946E092F982A982FEF3FEFC9016C
:10402000DF91CF911F910F91FF90EF90DF90CF9094
:10403000BF90AF909F908F907F906F9008952F9832
:104040002A9820E030E0EBCFCF92DF92EF92FF9200
:104050000F931F93CF93DF9311982A982F988DE099
:10406000982F9A95F1F72A9A982F9A95F1F72F9A07
:104070008A95F1F784E49CE00E946E09C7E1DEE0D6
:1040800015E002E080E4E82E8FE1F82EB0E8CB2EB8
:10409000BEE3DB2EDEC00A9A119A1298812F8A9510
:1040A000F1F71198812F8A95F1F7119A812F8A954E
:1040B000F1F71298812F8A95F1F71198812F8A953F
:1040C000F1F7119A812F8A95F1F71298812F8A952D
:1040D000F1F71198812F8A95F1F7119A812F8A951E
:1040E000F1F7129A812F8A95F1F71198812F8A950D
:1040F000F1F7119A812F8A95F1F71298812F8A95FD
:10410000F1F71198812F8A95F1F7119A812F8A95ED
:10411000F1F7129811980A98802F8A95F1F7C70144
:104120000197F1F70A9A119A129A812F8A95F1F75D
:104130001198812F8A95F1F7119A812F8A95F1F7BD
:104140001298812F8A95F1F71198812F8A95F1F7AE
:10415000119A812F8A95F1F7129A812F8A95F1F79A
:104160001198812F8A95F1F7119A812F8A95F1F78D
:104170001298812F8A95F1F71198812F8A95F1F77E
:10418000119A812F8A95F1F71298812F8A95F1F76C
:104190001198812F8A95F1F7119A812F8A95F1F75D
:1041A000129811980A98802F8A95F1F70E94CF1BD8
:1041B00090E0288130E08217930709F0E3C00A9A63
:1041C000119A1298812F8A95F1F71198812F8A956B
:1041D000F1F7119A812F8A95F1F7129A812F8A951A
:1041E000F1F71198812F8A95F1F7119A812F8A950D
:1041F000F1F7129A812F8A95F1F71198812F8A95FC
:10420000F1F7119A812F8A95F1F71298812F8A95EB
:10421000F1F71198812F8A95F1F7119A812F8A95DC
:10422000F1F71298812F8A95F1F71198812F8A95CD
:10423000F1F7119A812F8A95F1F7129811980A983F
:10424000802F8A95F1F721968EE0C739D80709F4B7
:10425000ABC088818F3F09F4B2CF0A9A119A129AA3
:10426000912F9A95F1F71198912F9A95F1F7119A4C
:10427000912F9A95F1F7129A912F9A95F1F711983B
:10428000912F9A95F1F7119A912F9A95F1F712982B
:10429000912F9A95F1F71198912F9A95F1F7119A1C
:1042A000912F9A95F1F71298912F9A95F1F711980D
:1042B000912F9A95F1F7119A912F9A95F1F71298FB
:1042C000912F9A95F1F71198912F9A95F1F7119AEC
:1042D000912F9A95F1F7129811980A98902F9A9524
:1042E000F1F790E00E941D1D80910A068D538230E7
:1042F00008F0D1CE0A9A119A1298812F8A95F1F777
:104300001198812F8A95F1F7119A812F8A95F1F7EB
:104310001298812F8A95F1F71198812F8A95F1F7DC
:10432000119A812F8A95F1F71298812F8A95F1F7CA
:104330001198812F8A95F1F7119A812F8A95F1F7BB
:10434000129A812F8A95F1F71198812F8A95F1F7AA
:10435000119A812F8A95F1F7129A812F8A95F1F798
:104360001198812F8A95F1F7119A812F8A95F1F78B
:10437000129811980A98802F8A95F1F7C601019733
:10438000F1F7D0CE87E19CE00E946E092F982A9821
:104390002FEF3FEFC901DF91CF911F910F91FF9058
:1043A000EF90DF90CF9008952F982A9820E030E08A
:1043B000F1CF8F929F92AF92BF92CF92DF92EF9206
:1043C000FF920F931F93DF93CF93CDB7DEB72A975A
:1043D0000FB6F894DEBF0FBECDBF11982A982F9864
:1043E0008DE0982F9A95F1F72A9A982F9A95F1F7E0
:1043F0002F9A8A95F1F70A9A119A129885E0982FC8
:104400009A95F1F71198982F9A95F1F7119A982F9C
:104410009A95F1F7129A982F9A95F1F71198982F8B
:104420009A95F1F7119A982F9A95F1F71298982F7B
:104430009A95F1F71198982F9A95F1F7119A982F6C
:104440009A95F1F71298982F9A95F1F71198982F5D
:104450009A95F1F7119A982F9A95F1F71298982F4B
:104460009A95F1F71198982F9A95F1F7119A8A95E4
:10447000F1F7129811980A9882E08A95F1F780E096
:1044800090E00E941D1DEE24FF2471E1872E72E052
:10449000972E5E010894A11CB11C05E062E0D62EA7
:1044A00098C00A9A119A1298802F8A95F1F711985C
:1044B000802F8A95F1F7119A802F8A95F1F712983B
:1044C000802F8A95F1F71198802F8A95F1F7119A2C
:1044D000802F8A95F1F7129A802F8A95F1F711981B
:1044E000802F8A95F1F7119A802F8A95F1F712980B
:1044F000802F8A95F1F71198802F8A95F1F7119AFC
:10450000802F8A95F1F71298802F8A95F1F71198EC
:10451000802F8A95F1F7119A802F8A95F1F71298DA
:1045200011980A988D2D8A95F1F70E94CF1B192FAB
:104530000E948D09812F0E948D090A9A119A129862
:10454000802F8A95F1F71198802F8A95F1F7119AAB
:10455000802F8A95F1F7129A802F8A95F1F711989A
:10456000802F8A95F1F7119A802F8A95F1F7129A88
:10457000802F8A95F1F71198802F8A95F1F7119A7B
:10458000802F8A95F1F71298802F8A95F1F711986C
:10459000802F8A95F1F7119A802F8A95F1F712985A
:1045A000802F8A95F1F71198802F8A95F1F7119A4B
:1045B000802F8A95F1F7129811980A988D2D8A9577
:1045C000F1F70894E11CF11C90E0E91694E0F9067B
:1045D00009F1C7018F709070892B09F062CF89EFC4
:1045E00099E00E946E09C701880F991F9F938F93CE
:1045F0009F928F92BF92AF920E94DD38C5010E94B8
:1046000055098DB79EB706960FB6F8949EBF0FBE9C
:104610008DBF47CF2F982A9811982A982F988DE010
:10462000982F9A95F1F72A9A982F9A95F1F72F9A41
:104630008A95F1F780EF99E00E946E09EE24FF243D
:1046400041E1842E42E0942E5E010894A11CB11C2D
:1046500015E002E097C00A9A119A129A35E0D32E1B
:10466000812F8A95F1F71198812F8A95F1F7119A88
:10467000812F8A95F1F71298812F8A95F1F7119879
:10468000812F8A95F1F7119A812F8A95F1F7129A65
:10469000812F8A95F1F71198812F8A95F1F7119A58
:1046A000812F8A95F1F71298812F8A95F1F7119849
:1046B000812F8A95F1F7119A812F8A95F1F7129837
:1046C000812F8A95F1F71198812F8A95F1F7119A28
:1046D000812F8A95F1F7129811980A9822E0C22E3C
:1046E000802F8A95F1F70E94CF1B0E948D090A9AAC
:1046F000119A1298812F8A95F1F71198812F8A9536
:10470000F1F7119A812F8A95F1F7129A812F8A95E4
:10471000F1F71198812F8A95F1F7119A812F8A95D7
:10472000F1F7129A812F8A95F1F71198812F8A95C6
:10473000F1F7119A812F8A95F1F71298812F8A95B6
:10474000F1F71198812F8A95F1F7119A812F8A95A7
:10475000F1F71298812F8A95F1F71198812F8A9598
:10476000F1F7119A812F8A95F1F7129811980A980A
:10477000802F8A95F1F70894E11CF11C90E8E91666
:10478000F104F1F0C7018F719070892B09F063CFAC
:104790008EEE99E00E946E09FF92EF929F928F92A7
:1047A000BF92AF920E94DD38C5010E9455098DB7B6
:1047B0009EB706960FB6F8949EBF0FBE8DBF4BCF27
:1047C0002F982A9811982A982F988DE0982F9A95CB
:1047D000F1F72A9A982F9A95F1F72F9A8A95F1F77F
:1047E0000A9A119A129805E08D2D8A95F1F7119881
:1047F0008D2D8A95F1F7119A8D2D8A95F1F71298E2
:104800008D2D8A95F1F711988D2D8A95F1F7119AD2
:104810008D2D8A95F1F712988D2D8A95F1F71198C3
:104820008D2D8A95F1F7119A8D2D8A95F1F71298B1
:104830008D2D8A95F1F711988D2D8A95F1F7119AA2
:104840008D2D8A95F1F712988D2D8A95F1F7119893
:104850008D2D8A95F1F7119A8D2D8A95F1F7129881
:1048600011980A9892E0F92E8C2D8A95F1F78FEF26
:104870009FE30E941D1D81EE99E00E946E090A9A35
:10488000119A12988D2D8A95F1F711988D2D8A9590
:10489000F1F7119A8D2D8A95F1F712988D2D8A9541
:1048A000F1F711988D2D8A95F1F7119A8D2D8A9532
:1048B000F1F7129A8D2D8A95F1F711988D2D8A9521
:1048C000F1F7119A8D2D8A95F1F712988D2D8A9511
:1048D000F1F711988D2D8A95F1F7119A8D2D8A9502
:1048E000F1F712988D2D8A95F1F711988D2D8A95F3
:1048F000F1F7119A8D2D8A95F1F7129811980A986F
:104900008C2D8A95F1F70E94CF1B192F0E948D09DB
:10491000812F0E948D090A9A119A12988D2D8A95DD
:10492000F1F711988D2D8A95F1F7119A8D2D8A95B1
:10493000F1F7129A8D2D8A95F1F711988D2D8A95A0
:10494000F1F7119A8D2D8A95F1F7129A8D2D8A958E
:10495000F1F711988D2D8A95F1F7119A8D2D8A9581
:10496000F1F712988D2D8A95F1F711988D2D8A9572
:10497000F1F7119A8D2D8A95F1F712988D2D8A9560
:10498000F1F711988D2D8A95F1F7119A8D2D8A9551
:10499000F1F7129811980A988C2D8A95F1F70A9AD6
:1049A000119A12988D2D8A95F1F711988D2D8A956F
:1049B000F1F7119A8D2D8A95F1F712988D2D8A9520
:1049C000F1F711988D2D8A95F1F7119A8D2D8A9511
:1049D000F1F7129A8D2D8A95F1F711988D2D8A9500
:1049E000F1F7119A8D2D8A95F1F712988D2D8A95F0
:1049F000F1F711988D2D8A95F1F7119A8D2D8A95E1
:104A0000F1F712988D2D8A95F1F711988D2D8A95D1
:104A1000F1F7119A8D2D8A95F1F7129811980A984D
:104A20008C2D8A95F1F70E94CF1B192F0E948D09BA
:104A3000812F0E948D090A9A119A12988D2D8A95BC
:104A4000F1F711988D2D8A95F1F7119A8D2D8A9590
:104A5000F1F7129A8D2D8A95F1F711988D2D8A957F
:104A6000F1F7119A8D2D8A95F1F7129A8D2D8A956D
:104A7000F1F711988D2D8A95F1F7119A8D2D8A9560
:104A8000F1F712988D2D8A95F1F711988D2D8A9551
:104A9000F1F7119A8D2D8A95F1F712988D2D8A953F
:104AA000F1F711988D2D8A95F1F7119A8D2D8A9530
:104AB000F1F7129811980A988C2D8A95F1F70A9AB5
:104AC000119A12988D2D8A95F1F711988D2D8A954E
:104AD000F1F7119A8D2D8A95F1F712988D2D8A95FF
:104AE000F1F711988D2D8A95F1F7119A8D2D8A95F0
:104AF000F1F7129A8D2D8A95F1F711988D2D8A95DF
:104B0000F1F7119A8D2D8A95F1F712988D2D8A95CE
:104B1000F1F711988D2D8A95F1F7119A8D2D8A95BF
:104B2000F1F712988D2D8A95F1F711988D2D8A95B0
:104B3000F1F7119A8D2D8A95F1F7129811980A982C
:104B40008C2D8A95F1F70E94CF1B192F0E948D0999
:104B5000812F0E948D090A9A119A12988D2D8A959B
:104B6000F1F711988D2D8A95F1F7119A8D2D8A956F
:104B7000F1F7129A8D2D8A95F1F711988D2D8A955E
:104B8000F1F7119A8D2D8A95F1F7129A8D2D8A954C
:104B9000F1F711988D2D8A95F1F7119A8D2D8A953F
:104BA000F1F712988D2D8A95F1F711988D2D8A9530
:104BB000F1F7119A8D2D8A95F1F712988D2D8A951E
:104BC000F1F711988D2D8A95F1F7119A8D2D8A950F
:104BD000F1F7129811980A988C2D8A95F1F70A9A94
:104BE000119A12988D2D8A95F1F711988D2D8A952D
:104BF000F1F7119A8D2D8A95F1F712988D2D8A95DE
:104C0000F1F711988D2D8A95F1F7119A8D2D8A95CE
:104C1000F1F7129A8D2D8A95F1F711988D2D8A95BD
:104C2000F1F7119A8D2D8A95F1F712988D2D8A95AD
:104C3000F1F711988D2D8A95F1F7119A8D2D8A959E
:104C4000F1F712988D2D8A95F1F711988D2D8A958F
:104C5000F1F7119A8D2D8A95F1F7129811980A980B
:104C60008C2D8A95F1F70E94CF1B192F0E948D0978
:104C7000812F0E948D090A9A119A12988D2D8A957A
:104C8000F1F711988D2D8A95F1F7119A8D2D8A954E
:104C9000F1F7129A8D2D8A95F1F711988D2D8A953D
:104CA000F1F7119A8D2D8A95F1F7129A8D2D8A952B
:104CB000F1F711988D2D8A95F1F7119A8D2D8A951E
:104CC000F1F712988D2D8A95F1F711988D2D8A950F
:104CD000F1F7119A8D2D8A95F1F712988D2D8A95FD
:104CE000F1F711988D2D8A95F1F7119A8D2D8A95EE
:104CF000F1F7129811980A988C2D8A95F1F70A9A73
:104D0000119A12988D2D8A95F1F711988D2D8A950B
:104D1000F1F7119A8D2D8A95F1F7129A8D2D8A95BA
:104D2000F1F711988D2D8A95F1F7119A8D2D8A95AD
:104D3000F1F7129A8D2D8A95F1F711988D2D8A959C
:104D4000F1F7119A8D2D8A95F1F712988D2D8A958C
:104D5000F1F711988D2D8A95F1F7119A8D2D8A957D
:104D6000F1F712988D2D8A95F1F711988D2D8A956E
:104D7000F1F7119A8D2D8A95F1F7129811980A98EA
:104D80008C2D8A95F1F70A9A119A12988D2D8A9591
:104D9000F1F711988D2D8A95F1F7119A8D2D8A953D
:104DA000F1F7129A802F8A95F1F71198802F8A9542
:104DB000F1F7119A802F8A95F1F7129A802F8A9530
:104DC000F1F71198802F8A95F1F7119A802F8A9523
:104DD000F1F71298802F8A95F1F71198802F8A9514
:104DE000F1F7119A802F8A95F1F71298802F8A9502
:104DF000F1F71198802F8A95F1F7119A802F8A95F3
:104E0000F1F7129811980A988F2D8A95F1F70A9A5E
:104E1000119A1298802F8A95F1F71198802F8A9510
:104E2000F1F7119A802F8A95F1F7129A802F8A95BF
:104E3000F1F71198802F8A95F1F7119A802F8A95B2
:104E4000F1F7129A802F8A95F1F71198802F8A95A1
:104E5000F1F7119A802F8A95F1F71298802F8A9591
:104E6000F1F71198802F8A95F1F7119A802F8A9582
:104E7000F1F71298802F8A95F1F71198802F8A9573
:104E8000F1F7119A802F8A95F1F7129811980A98E4
:104E90008F2D8A95F1F780ED99E00E946E090A9AAC
:104EA000119A1298802F8A95F1F71198802F8A9580
:104EB000F1F7119A802F8A95F1F71298802F8A9531
:104EC000F1F71198802F8A95F1F7119A802F8A9522
:104ED000F1F7129A802F8A95F1F71198802F8A9511
:104EE000F1F7119A802F8A95F1F71298802F8A9501
:104EF000F1F71198802F8A95F1F7119A802F8A95F2
:104F0000F1F71298802F8A95F1F71198802F8A95E2
:104F1000F1F7119A0A95F1F7129811980A98FA94F4
:104F2000F1F70E94CF1B192F0E948D09812F0E943B
:104F30008D092F982A982A960FB6F894DEBF0FBED7
:104F4000CDBFCF91DF911F910F91FF90EF90DF9038
:104F5000CF90BF90AF909F908F9008950F931F9325
:104F6000DF93CF930F92CDB7DEB711982A982F9881
:104F70008DE0982F9A95F1F72A9A982F9A95F1F744
:104F80002F9A8A95F1F70A9A119A129815E0812FB3
:104F90008A95F1F71198812F8A95F1F7119A812F4F
:104FA0008A95F1F71298812F8A95F1F71198812F40
:104FB0008A95F1F7119A812F8A95F1F71298812F2E
:104FC0008A95F1F71198812F8A95F1F7119A812F1F
:104FD0008A95F1F71298812F8A95F1F71198812F10
:104FE0008A95F1F7119A812F8A95F1F71298812FFE
:104FF0008A95F1F71198812F8A95F1F7119A812FEF
:105000008A95F1F7129811980A9802E0802F8A95F4
:10501000F1F780E090E00E941D1D0A9A119A129803
:10502000812F8A95F1F71198812F8A95F1F7119ABE
:10503000812F8A95F1F7129A812F8A95F1F71198AD
:10504000812F8A95F1F7119A812F8A95F1F7129A9B
:10505000812F8A95F1F71198812F8A95F1F7119A8E
:10506000812F8A95F1F71298812F8A95F1F711987F
:10507000812F8A95F1F7119A812F8A95F1F712986D
:10508000812F8A95F1F71198812F8A95F1F7119A5E
:10509000812F8A95F1F7129811980A98802F8A9596
:1050A000F1F70A9A119A1298812F8A95F1F71198BF
:1050B000812F8A95F1F7119A812F8A95F1F7129A2B
:1050C000812F8A95F1F71198812F8A95F1F7119A1E
:1050D000812F8A95F1F7129A812F8A95F1F711980D
:1050E000812F8A95F1F7119A812F8A95F1F71298FD
:1050F000812F8A95F1F71198812F8A95F1F7119AEE
:10510000812F8A95F1F71298812F8A95F1F71198DE
:10511000812F8A95F1F7119A812F8A95F1F71298CC
:1051200011980A98802F8A95F1F70A9A119A129885
:10513000812F8A95F1F71198812F8A95F1F7119AAD
:10514000812F8A95F1F7129A812F8A95F1F711989C
:10515000812F8A95F1F7119A812F8A95F1F7129A8A
:10516000812F8A95F1F71198812F8A95F1F7119A7D
:10517000812F8A95F1F71298812F8A95F1F711986E
:10518000812F8A95F1F7119A812F8A95F1F712985C
:10519000812F8A95F1F71198812F8A95F1F7119A4D
:1051A000812F8A95F1F7129811980A98802F8A9585
:1051B000F1F70A9A119A1298812F8A95F1F71198AE
:1051C000812F8A95F1F7119A812F8A95F1F7129A1A
:1051D000812F8A95F1F71198812F8A95F1F7119A0D
:1051E000812F8A95F1F7129A812F8A95F1F71198FC
:1051F000812F8A95F1F7119A812F8A95F1F71298EC
:10520000812F8A95F1F71198812F8A95F1F7119ADC
:10521000812F8A95F1F71298812F8A95F1F71198CD
:10522000812F8A95F1F7119A812F8A95F1F71298BB
:1052300011980A98802F8A95F1F70A9A119A129874
:10524000812F8A95F1F71198812F8A95F1F7119A9C
:10525000812F8A95F1F7129A812F8A95F1F711988B
:10526000812F8A95F1F7119A812F8A95F1F7129A79
:10527000812F8A95F1F71198812F8A95F1F7119A6C
:10528000812F8A95F1F71298812F8A95F1F711985D
:10529000812F8A95F1F7119A812F8A95F1F712984B
:1052A000812F8A95F1F71198812F8A95F1F7119A3C
:1052B000812F8A95F1F7129811980A98802F8A9574
:1052C000F1F70A9A119A1298812F8A95F1F711989D
:1052D000812F8A95F1F7119A812F8A95F1F7129A09
:1052E000812F8A95F1F71198812F8A95F1F7119AFC
:1052F000812F8A95F1F7129A812F8A95F1F71198EB
:10530000812F8A95F1F7119A812F8A95F1F71298DA
:10531000812F8A95F1F71198812F8A95F1F7119ACB
:10532000812F8A95F1F71298812F8A95F1F71198BC
:10533000812F8A95F1F7119A812F8A95F1F71298AA
:1053400011980A98802F8A95F1F70A9A119A129863
:10535000812F8A95F1F71198812F8A95F1F7119A8B
:10536000812F8A95F1F71298812F8A95F1F711987C
:10537000812F8A95F1F7119A812F8A95F1F7129A68
:10538000812F8A95F1F71198812F8A95F1F7119A5B
:10539000812F8A95F1F71298812F8A95F1F711984C
:1053A000812F8A95F1F7119A812F8A95F1F712983A
:1053B000812F8A95F1F71198812F8A95F1F7119A2B
:1053C0001A95F1F7129811980A980A95F1F70E9428
:1053D000CF1B8C0116950795129502950F7001272A
:1053E0001F70012710700238110509F46BC00338D3
:1053F0001105D0F00338110509F446C0083811052D
:1054000041F18BEF99E00E946E0980E00E948D09C6
:10541000802F09830E948D099981892F0F90CF9148
:10542000DF911F910F9108950D331105E1F10E33B6
:10543000110539F78AE19AE00E946E098EE38093A4
:105440000A069EE3892F0F90CF91DF911F910F9154
:10545000089588E29BE00E946E0987ED9AE00E9421
:105460006E0989EB9AE00E946E098CE69AE00E9430
:105470006E0988E880930A0698E8892F0F90CF91EB
:10548000DF911F910F91089582E49AE00E946E09C6
:1054900083E880930A0693E8892F0F90CF91DF91DC
:1054A0001F910F9108958EE29AE00E946E098DE39C
:1054B00080930A069DE3892F0F90CF91DF911F9172
:1054C0000F91089587E59AE00E946E0982E8809323
:1054D0000A0692E8892F0F90CF91DF911F910F91CB
:1054E00008952F923F925F926F927F928F929F9238
:1054F000AF92BF92CF92DF92EF92FF920F931F93E2
:10550000CF93DF9380EF9BE00E946E0911982A9859
:105510002F988DE0982F9A95F1F72A9A982F9A95BF
:10552000F1F72F9A8A95F1F70A9A119A129885E065
:10553000982F9A95F1F71198982F9A95F1F7119A5B
:10554000982F9A95F1F71298982F9A95F1F711984C
:10555000982F9A95F1F7119A982F9A95F1F712983A
:10556000982F9A95F1F71198982F9A95F1F7119A2B
:10557000982F9A95F1F71298982F9A95F1F711981C
:10558000982F9A95F1F7119A982F9A95F1F712980A
:10559000982F9A95F1F71198982F9A95F1F7119AFB
:1055A0008A95F1F7129811980A9882E08A95F1F796
:1055B0008FEF9FE30E941D1DB7E9EB2EBEE0FB2E8F
:1055C0000CEF8824992415E0A2E05A2EF0E42F2E47
:1055D000FFE13F2EECC00A9A119A1298812F8A950A
:1055E000F1F71198812F8A95F1F7119A812F8A95F9
:1055F000F1F71298812F8A95F1F71198812F8A95EA
:10560000F1F7119A812F8A95F1F71298812F8A95D7
:10561000F1F71198812F8A95F1F7119A812F8A95C8
:10562000F1F7129A812F8A95F1F71198812F8A95B7
:10563000F1F7119A812F8A95F1F71298812F8A95A7
:10564000F1F71198812F8A95F1F7119A812F8A9598
:10565000F1F7129811980A98852D8A95F1F7C101F2
:105660000197F1F70A9A119A1298812F8A95F1F70A
:105670001198812F8A95F1F7119A812F8A95F1F768
:105680001298812F8A95F1F71198812F8A95F1F759
:10569000119A812F8A95F1F7129A812F8A95F1F745
:1056A0001198812F8A95F1F7119A812F8A95F1F738
:1056B0001298812F8A95F1F71198812F8A95F1F729
:1056C000119A812F8A95F1F71298812F8A95F1F717
:1056D0001198812F8A95F1F7119A812F8A95F1F708
:1056E000129811980A98852D8A95F1F70E94CF1B80
:1056F000EC01F701B180AA24C50180709F7320815D
:1057000030E0822B932B9E013F732817390709F055
:1057100011C10A9A119A1298812F8A95F1F711985E
:10572000812F8A95F1F7119A812F8A95F1F7129AB4
:10573000812F8A95F1F71198812F8A95F1F7119AA7
:10574000812F8A95F1F7129A812F8A95F1F7119896
:10575000812F8A95F1F7119A812F8A95F1F7129886
:10576000812F8A95F1F71198812F8A95F1F7119A77
:10577000812F8A95F1F71298812F8A95F1F7119868
:10578000812F8A95F1F7119A812F8A95F1F7129856
:1057900011980A98852D8A95F1F70F5F82E090E0C5
:1057A000880E991EE80EF91E043009F4ACC00330CF
:1057B00008F4AFCF34010894611C711CF701D1804B
:1057C000CC24960120703F73808190E0282B392BE8
:1057D000FFE32F3F3F0709F49CCF0A9A119A1298D2
:1057E000812F8A95F1F71198812F8A95F1F7119AF7
:1057F000812F8A95F1F7129A812F8A95F1F71198E6
:10580000812F8A95F1F7119A812F8A95F1F71298D5
:10581000812F8A95F1F71198812F8A95F1F7119AC6
:10582000812F8A95F1F71298812F8A95F1F71198B7
:10583000812F8A95F1F7119A812F8A95F1F71298A5
:10584000812F8A95F1F71198812F8A95F1F7119A96
:10585000812F8A95F1F7129811980A98852D8A95CB
:10586000F1F7C9010E941D1D80910A068D538230F7
:1058700008F0B1CE0A9A119A1298812F8A95F1F701
:105880001198812F8A95F1F7119A812F8A95F1F756
:105890001298812F8A95F1F71198812F8A95F1F747
:1058A000119A812F8A95F1F71298812F8A95F1F735
:1058B0001198812F8A95F1F7119A812F8A95F1F726
:1058C000129A812F8A95F1F71198812F8A95F1F715
:1058D000119A812F8A95F1F71298812F8A95F1F705
:1058E0001198812F8A95F1F7119A812F8A95F1F7F6
:1058F000129811980A98852D8A95F1F780E995E616
:105900000197F1F7AFCE2F982A9820E030E0C90137
:10591000DF91CF911F910F91FF90EF90DF90CF908B
:10592000BF90AF909F908F907F906F905F903F90CF
:105930002F9008958AEB9BE00E946E0981EB9BE01B
:105940000E946E0987E99EE0680E791EF30180814E
:105950000E948D0987E99EE0880E991EF4018081DE
:105960000E948D0988EA9BE00E946E098D2F0E949B
:105970008D098C2F0E948D0989E69BE00E946E099B
:105980008DE39BE00E946E092F982A982FEF3FEF3E
:10599000BECF0F931F9387E999E00E946E0911987B
:1059A0002A982F988DE0982F9A95F1F72A9A982F98
:1059B0009A95F1F72F9A8A95F1F780910A068D53FF
:1059C000823008F495C00A9A119A129815E0812F36
:1059D0008A95F1F71198812F8A95F1F7119A812F05
:1059E0008A95F1F71298812F8A95F1F71198812FF6
:1059F0008A95F1F7119A812F8A95F1F71298812FE4
:105A00008A95F1F71198812F8A95F1F7119A812FD4
:105A10008A95F1F71298812F8A95F1F71198812FC5
:105A20008A95F1F7119A812F8A95F1F71298812FB3
:105A30008A95F1F71198812F8A95F1F7119A812FA4
:105A40008A95F1F7129811980A9802E0802F8A95AA
:105A5000F1F78FEF9FE30E941D1D0A9A119A129A87
:105A6000812F8A95F1F71198812F8A95F1F7119A74
:105A7000812F8A95F1F71298812F8A95F1F7119865
:105A8000812F8A95F1F7119A812F8A95F1F7129853
:105A9000812F8A95F1F71198812F8A95F1F7119A44
:105AA000812F8A95F1F7129A812F8A95F1F7119833
:105AB000812F8A95F1F7119A812F8A95F1F7129823
:105AC000812F8A95F1F71198812F8A95F1F7119A14
:105AD0001A95F1F7129811980A980A95F1F780EE45
:105AE0009EE20197F1F72F982A981F910F91089540
:105AF0000A9A119A129815E0812F8A95F1F7119858
:105B0000812F8A95F1F7119A812F8A95F1F71298D2
:105B1000812F8A95F1F71198812F8A95F1F7119AC3
:105B2000812F8A95F1F71298812F8A95F1F71198B4
:105B3000812F8A95F1F7119A812F8A95F1F71298A2
:105B4000812F8A95F1F71198812F8A95F1F7119A93
:105B5000812F8A95F1F71298812F8A95F1F7119884
:105B6000812F8A95F1F7119A812F8A95F1F7129872
:105B700011980A9802E0802F8A95F1F78FEF9FE342
:105B80000E941D1D0A9A119A1298812F8A95F1F789
:105B90001198812F8A95F1F7119A812F8A95F1F743
:105BA000129A812F8A95F1F71198812F8A95F1F732
:105BB000119A812F8A95F1F7129A812F8A95F1F720
:105BC0001198812F8A95F1F7119A812F8A95F1F713
:105BD0001298812F8A95F1F71198812F8A95F1F704
:105BE000119A812F8A95F1F71298812F8A95F1F7F2
:105BF0001198812F8A95F1F7119A812F8A95F1F7E3
:105C0000129811980A98802F8A95F1F70A9A119A9A
:105C10001298812F8A95F1F71198812F8A95F1F7C3
:105C2000119A812F8A95F1F7129A812F8A95F1F7AF
:105C30001198812F8A95F1F7119A812F8A95F1F7A2
:105C4000129A812F8A95F1F71198812F8A95F1F791
:105C5000119A812F8A95F1F71298812F8A95F1F781
:105C60001198812F8A95F1F7119A812F8A95F1F772
:105C70001298812F8A95F1F71198812F8A95F1F763
:105C8000119A812F8A95F1F7129811980A98802F0E
:105C90008A95F1F70A9A119A1298812F8A95F1F74D
:105CA0001198812F8A95F1F7119A812F8A95F1F732
:105CB000129A812F8A95F1F71198812F8A95F1F721
:105CC000119A812F8A95F1F7129A812F8A95F1F70F
:105CD0001198812F8A95F1F7119A812F8A95F1F702
:105CE0001298812F8A95F1F71198812F8A95F1F7F3
:105CF000119A812F8A95F1F71298812F8A95F1F7E1
:105D00001198812F8A95F1F7119A812F8A95F1F7D1
:105D1000129811980A98802F8A95F1F70A9A119A89
:105D20001298812F8A95F1F71198812F8A95F1F7B2
:105D3000119A812F8A95F1F7129A812F8A95F1F79E
:105D40001198812F8A95F1F7119A812F8A95F1F791
:105D5000129A812F8A95F1F71198812F8A95F1F780
:105D6000119A812F8A95F1F71298812F8A95F1F770
:105D70001198812F8A95F1F7119A812F8A95F1F761
:105D80001298812F8A95F1F71198812F8A95F1F752
:105D9000119A812F8A95F1F7129811980A98802FFD
:105DA0008A95F1F70A9A119A1298812F8A95F1F73C
:105DB0001198812F8A95F1F7119A812F8A95F1F721
:105DC000129A812F8A95F1F71198812F8A95F1F710
:105DD000119A812F8A95F1F7129A812F8A95F1F7FE
:105DE0001198812F8A95F1F7119A812F8A95F1F7F1
:105DF0001298812F8A95F1F71198812F8A95F1F7E2
:105E0000119A812F8A95F1F71298812F8A95F1F7CF
:105E10001198812F8A95F1F7119A812F8A95F1F7C0
:105E2000129811980A98802F8A95F1F70A9A119A78
:105E30001298812F8A95F1F71198812F8A95F1F7A1
:105E4000119A812F8A95F1F7129A812F8A95F1F78D
:105E50001198812F8A95F1F7119A812F8A95F1F780
:105E6000129A812F8A95F1F71198812F8A95F1F76F
:105E7000119A812F8A95F1F71298812F8A95F1F75F
:105E80001198812F8A95F1F7119A812F8A95F1F750
:105E90001298812F8A95F1F71198812F8A95F1F741
:105EA000119A812F8A95F1F7129811980A98802FEC
:105EB0008A95F1F70A9A119A1298812F8A95F1F72B
:105EC0001198812F8A95F1F7119A812F8A95F1F710
:105ED000129A812F8A95F1F71198812F8A95F1F7FF
:105EE000119A812F8A95F1F7129A812F8A95F1F7ED
:105EF0001198812F8A95F1F7119A812F8A95F1F7E0
:105F00001298812F8A95F1F71198812F8A95F1F7D0
:105F1000119A812F8A95F1F71298812F8A95F1F7BE
:105F20001198812F8A95F1F7119A812F8A95F1F7AF
:105F3000129811980A98802F8A95F1F70A9A119A67
:105F4000129A812F8A95F1F71198812F8A95F1F78E
:105F5000119A812F8A95F1F71298812F8A95F1F77E
:105F60001198812F8A95F1F7119A812F8A95F1F76F
:105F70001298812F8A95F1F71198812F8A95F1F760
:105F8000119A812F8A95F1F71298812F8A95F1F74E
:105F90001198812F8A95F1F7119A812F8A95F1F73F
:105FA0001298812F8A95F1F71198812F8A95F1F730
:105FB000119A812F8A95F1F7129811980A98802FDB
:105FC0008A95F1F70A9A119A129A812F8A95F1F718
:105FD0001198812F8A95F1F7119A812F8A95F1F7FF
:105FE000129A812F8A95F1F71198812F8A95F1F7EE
:105FF000119A812F8A95F1F7129A812F8A95F1F7DC
:106000001198812F8A95F1F7119A812F8A95F1F7CE
:106010001298812F8A95F1F71198812F8A95F1F7BF
:10602000119A812F8A95F1F71298812F8A95F1F7AD
:106030001198812F8A95F1F7119A812F8A95F1F79E
:10604000129811980A98802F8A95F1F70A9A119A56
:106050001298812F8A95F1F71198812F8A95F1F77F
:10606000119A812F8A95F1F71298812F8A95F1F76D
:106070001198812F8A95F1F7119A812F8A95F1F75E
:106080001298812F8A95F1F71198812F8A95F1F74F
:10609000119A812F8A95F1F7129A812F8A95F1F73B
:1060A0001198812F8A95F1F7119A812F8A95F1F72E
:1060B0001298812F8A95F1F71198812F8A95F1F71F
:1060C000119A812F8A95F1F7129811980A98802FCA
:1060D0008A95F1F780E995E60197F1F70A9A119A06
:1060E000129A812F8A95F1F71198812F8A95F1F7ED
:1060F000119A812F8A95F1F71298812F8A95F1F7DD
:106100001198812F8A95F1F7119A812F8A95F1F7CD
:106110001298812F8A95F1F71198812F8A95F1F7BE
:10612000119A812F8A95F1F71298812F8A95F1F7AC
:106130001198812F8A95F1F7119A812F8A95F1F79D
:106140001298812F8A95F1F71198812F8A95F1F78E
:10615000119A812F8A95F1F7129811980A98802F39
:106160008A95F1F70A9A119A129A812F8A95F1F776
:106170001198812F8A95F1F7119A812F8A95F1F75D
:10618000129A812F8A95F1F71198812F8A95F1F74C
:10619000119A812F8A95F1F7129A812F8A95F1F73A
:1061A0001198812F8A95F1F7119A812F8A95F1F72D
:1061B0001298812F8A95F1F71198812F8A95F1F71E
:1061C000119A812F8A95F1F71298812F8A95F1F70C
:1061D0001198812F8A95F1F7119A1A95F1F7129873
:1061E00011980A980A95F1F72F982A981F910F9104
:1061F00008950F931F9311982A982F988DE0982F48
:106200009A95F1F72A9A982F9A95F1F72F9A8A95ED
:10621000F1F78EEE9CE00E946E090A9A119A12988C
:1062200015E0812F8A95F1F71198812F8A95F1F762
:10623000119A812F8A95F1F7129A812F8A95F1F799
:106240001198812F8A95F1F7119A812F8A95F1F78C
:106250001298812F8A95F1F71198812F8A95F1F77D
:10626000119A812F8A95F1F71298812F8A95F1F76B
:106270001198812F8A95F1F7119A812F8A95F1F75C
:106280001298812F8A95F1F71198812F8A95F1F74D
:10629000119A812F8A95F1F7129811980A9802E0C5
:1062A000802F8A95F1F78FEF9FE30E941D1D0A9AB8
:1062B000119A129A812F8A95F1F71198812F8A9558
:1062C000F1F7119A812F8A95F1F71298812F8A950B
:1062D000F1F71198812F8A95F1F7119A812F8A95FC
:1062E000F1F71298812F8A95F1F71198812F8A95ED
:1062F000F1F7119A812F8A95F1F7129A812F8A95D9
:10630000F1F71198812F8A95F1F7119A812F8A95CB
:10631000F1F71298812F8A95F1F71198812F8A95BC
:10632000F1F7119A812F8A95F1F7129811980A982E
:10633000802F8A95F1F780910A068D53823008F4F8
:10634000E9C080EE9EE20197F1F782ED9CE00E94A9
:106350006E090A9A119A129815E0812F8A95F1F721
:106360001198812F8A95F1F7119A812F8A95F1F76B
:10637000129A812F8A95F1F71198812F8A95F1F75A
:10638000119A812F8A95F1F71298812F8A95F1F74A
:106390001198812F8A95F1F7119A812F8A95F1F73B
:1063A0001298812F8A95F1F71198812F8A95F1F72C
:1063B000119A812F8A95F1F71298812F8A95F1F71A
:1063C0001198812F8A95F1F7119A812F8A95F1F70B
:1063D000129811980A9802E0802F8A95F1F78FEFB2
:1063E0009FE30E941D1D0A9A119A129A812F8A9585
:1063F000F1F71198812F8A95F1F7119A812F8A95DB
:10640000F1F7129A812F8A95F1F71198812F8A95C9
:10641000F1F7119A812F8A95F1F71298812F8A95B9
:10642000F1F71198812F8A95F1F7119A812F8A95AA
:10643000F1F7129A812F8A95F1F71198812F8A9599
:10644000F1F7119A812F8A95F1F71298812F8A9589
:10645000F1F71198812F8A95F1F7119A812F8A957A
:10646000F1F7129811980A98802F8A95F1F7809188
:106470000A068D53823048F080EE9EE20197F1F7D4
:106480002F982A981F910F9108950A9A119A12989D
:10649000812F8A95F1F71198812F8A95F1F7119A3A
:1064A000812F8A95F1F71298812F8A95F1F711982B
:1064B000812F8A95F1F7119A812F8A95F1F7129819
:1064C000812F8A95F1F71198812F8A95F1F7119A0A
:1064D000812F8A95F1F7129A812F8A95F1F71198F9
:1064E000812F8A95F1F7119A812F8A95F1F7129AE7
:1064F000812F8A95F1F71198812F8A95F1F7119ADA
:10650000812F8A95F1F7129811980A98802F8A9511
:10651000F1F7B2CF0A9A119A1298812F8A95F1F762
:106520001198812F8A95F1F7119A812F8A95F1F7A9
:106530001298812F8A95F1F71198812F8A95F1F79A
:10654000119A812F8A95F1F71298812F8A95F1F788
:106550001198812F8A95F1F7119A812F8A95F1F779
:10656000129A812F8A95F1F71198812F8A95F1F768
:10657000119A812F8A95F1F7129A812F8A95F1F756
:106580001198812F8A95F1F7119A812F8A95F1F749
:10659000129811980A98802F8A95F1F7D2CEEF922F
:1065A000FF920F931F937B018C0120E030E040E0CD
:1065B0005FE40E94CF3588238CF020E030E040E09B
:1065C0005FE4C801B7010E9447340E948D369B01E9
:1065D000AC01205030404040504806C0C801B701CF
:1065E0000E948D369B01AC01B901CA011F910F9128
:1065F000FF90EF900895A0E0B0E0E1E0F3E30C94A9
:10660000A63BDC012B01FA019C91923008F439C1C0
:10661000EB018881823008F433C1943069F484300E
:1066200009F02FC111969C9111978981981709F44F
:1066300028C1A9E1B2E025C1843009F421C182302A
:10664000A9F4923009F01DC19A01AD0188E0EA0178
:106650000990AE01E90109929E018150C1F7E20162
:10666000898111969C918923818308C1923009F414
:1066700007C112962D903C901397EB018A819B8164
:106680001496AD90BD90CD90DC901797EC80FD8076
:106690000E811F819101281B390BB90137FF04C0FE
:1066A00066277727621B730B603271050CF061C09F
:1066B000121613066CF537014801062E04C0969495
:1066C0008794779467940A94D2F721E030E040E011
:1066D00050E004C0220F331F441F551F6A95D2F7A4
:1066E00021503040404050402E213F214023512333
:1066F000211531054105510521F021E030E040E050
:1067000050E079018A01E628F728082919293CC0B8
:10671000232BD1F1260E371E35014601062E04C06B
:1067200096948794779467940A94D2F721E030E0A6
:1067300040E050E004C0220F331F441F551F6A95EC
:10674000D2F721503040404050402A213B214C217B
:106750005D21211531054105510521F021E030E091
:1067600040E050E059016A01A628B728C828D92876
:106770000BC0821593052CF01C01AA24BB246501D3
:1067800003C0EE24FF24870111969C91D20111963B
:106790008C91981709F445C0992339F0A801970105
:1067A0002A193B094C095D0906C0A60195012E195D
:1067B0003F09400B510B57FD08C0118233822282E2
:1067C00024833583468357831DC081E081833382D0
:1067D000228288279927DC01821B930BA40BB50B1F
:1067E00084839583A683B7830DC0220F331F441F74
:1067F000551F248335834683578382819381019774
:10680000938382832481358146815781DA01C901CE
:106810000197A109B1098F5F9F4FAF4FBF4328F385
:106820000BC0918333822282EA0CFB1C0C1D1D1DC0
:10683000E482F5820683178383E080832481358197
:106840004681578157FF1AC0C901AA2797FDA09515
:10685000BA2F81709070A070B0705695479537959B
:106860002795822B932BA42BB52B84839583A6830A
:10687000B78382819381019693838283DF0101C074
:10688000D201CD01CDB7DEB7E2E10C94C23BA0E26C
:10689000B0E0EDE4F4E30C94B23B69837A838B833C
:1068A0009C832D833E834F835887E9E0EE2EF12CA5
:1068B000EC0EFD1EB701CE0101960E9405388E0137
:1068C0000F5E1F4FB801CE0105960E9405388A89D8
:1068D00091E089278A8BAE01475E5F4FB801C701FF
:1068E0000E94FB320E943037A096E6E00C94CE3B2B
:1068F000A0E2B0E0EEE7F4E30C94B23B69837A8364
:106900008B839C832D833E834F835887F9E0EF2E42
:10691000F12CEC0EFD1EB701CE0101960E94053848
:106920008E010F5E1F4FB801CE0105960E940538FB
:10693000AE01475E5F4FB801C7010E94FB320E9463
:106940003037A096E6E00C94CE3BA0E2B0E0EBEA54
:10695000F4E30C94A63B69837A838B839C832D8319
:106960003E834F835887BE01675F7F4FCE010196FC
:106970000E940538BE016F5E7F4FCE0105960E94D2
:1069800005389985923088F089898230C8F0943032
:1069900019F4823051F404C0843029F4923081F427
:1069A00089E192E0C6C0923049F420E09A858A8954
:1069B000981321E02A87CE010996BBC0823049F4A2
:1069C00020E09A858A89981321E02A8BCE0141968E
:1069D000B0C02D843E844F8458886D887E888F880F
:1069E000988CEE24FF248701AA24BB24650140E093
:1069F00050E060E070E0E0E0F0E0C1018170907094
:106A0000892BE9F0E60CF71C081D191D9A01AB0152
:106A10002A0D3B1D4C1D5D1D80E090E0A0E0B0E024
:106A2000E614F7040805190520F481E090E0A0E0E1
:106A3000B0E0BA01A901480F591F6A1F7B1FAA0CB9
:106A4000BB1CCC1CDD1C97FE08C081E090E0A0E0E0
:106A5000B0E0A82AB92ACA2ADB2A3196E032F10529
:106A600049F0660C771C881C991C569447943794FF
:106A70002794C3CFFA85EA892B893C898B859C852D
:106A8000280F391F2E5F3F4F17C0CA0181709070C9
:106A9000892B61F016950795F794E79480E090E0D4
:106AA000A0E0B0E8E82AF92A0A2B1B2B7695679517
:106AB000579547952F5F3F4F77FDE7CF0CC0440FA9
:106AC000551F661F771F17FD4160EE0CFF1C001F4E
:106AD000111F21503040403090E0590790E0690785
:106AE00090E4790760F32B8F3C8FDB01CA018F772D
:106AF0009070A070B07080349105A105B10561F46B
:106B000047FD0AC0E114F1040105110529F0405CBC
:106B10005F4F6F4F7F4F40781A8EFE1711F081E064
:106B20008A8F4D8F5E8F6F8F78A383E0898FCE0120
:106B300049960E943037A096E2E10C94C23BA8E14E
:106B4000B0E0E5EAF5E30C94B23B69837A838B838A
:106B50009C832D833E834F83588789E0E82EF12C58
:106B6000EC0EFD1EB701CE0101960E9405388E0184
:106B70000F5E1F4FB801CE0105960E94053889852A
:106B8000823040F08989823028F0B801C7010E9424
:106B90007D3801C08FEF6896E6E00C94CE3BA8E10B
:106BA000B0E0E5EDF5E30C94B23B69837A838B8327
:106BB0009C832D833E834F83588789E0E82EF12CF8
:106BC000EC0EFD1EB701CE0101960E9405388E0124
:106BD0000F5E1F4FB801CE0105960E9405388985CA
:106BE000823040F08989823028F0B801C7010E94C4
:106BF0007D3801C08FEF6896E6E00C94CE3BA8E1AB
:106C0000B0E0E5E0F6E30C94B23B69837A838B83D2
:106C10009C832D833E834F83588789E0E82EF12C97
:106C2000EC0EFD1EB701CE0101960E9405388E01C3
:106C30000F5E1F4FB801CE0105960E940538898569
:106C4000823040F08989823028F0B801C7010E9463
:106C50007D3801C081E06896E6E00C94CE3BA8E068
:106C6000B0E0E5E3F6E30C94AF3B9B01AC0183E0BD
:106C70008983DA01C9018827B7FD83959927AA2757
:106C8000BB27B82E211531054105510519F482E0C5
:106C900089833AC08823A9F0203080E0380780E05B
:106CA000480780E8580729F460E070E080E09FEC36
:106CB00030C0EE24FF248701E21AF30A040B150BFF
:106CC00002C079018A018EE1C82ED12CDC82CB82F0
:106CD000ED82FE820F831887C801B7010E94E1365A
:106CE00001971816190684F4082E04C0EE0CFF1C38
:106CF000001F111F0A94D2F7ED82FE820F831887BE
:106D0000C81AD90ADC82CB82BA82CE0101960E94CF
:106D100030372896E9E00C94CB3BACE0B0E0E3E9F7
:106D2000F6E30C94B63B69837A838B839C83BE0124
:106D30006B5F7F4FCE0101960E9405388D818230B6
:106D400061F1823050F1843021F48E81882351F139
:106D50002EC02F81388537FD20C06E812F3131053F
:106D60001CF06623F9F023C08EE190E0821B930BA8
:106D700029853A854B855C8504C05695479537959E
:106D800027958A95D2F76623B1F0509540953095B6
:106D900021953F4F4F4F5F4F0EC020E030E040E065
:106DA00050E009C02FEF3FEF4FEF5FE704C020E056
:106DB00030E040E050E8B901CA012C96E2E00C94C2
:106DC000D23BEF92FF920F931F937B018C0180E0E7
:106DD000E81680E0F80681E0080780E0180788F4EC
:106DE0008FEFE816F1040105110531F028F088E075
:106DF00090E0A0E0B0E017C080E090E0A0E0B0E05C
:106E000012C080E0E81680E0F80680E0080781E024
:106E1000180728F088E190E0A0E0B0E004C080E12D
:106E200090E0A0E0B0E020E230E040E050E0281B3D
:106E3000390B4A0B5B0B04C016950795F794E79442
:106E40008A95D2F7F701EF5DFD4F8081281B31094C
:106E500041095109C9011F910F91FF90EF900895C9
:106E6000DF92EF92FF920F931F93FC01E480F58075
:106E700006811781D1808081823048F480E090E0E3
:106E8000A0E1B0E0E82AF92A0A2B1B2BA5C0843028
:106E900009F49FC0823021F4EE24FF24870105C04D
:106EA000E114F1040105110519F4E0E0F0E096C0E9
:106EB000628173819FEF623879070CF05BC022E832
:106EC0003FEF261B370B2A3131052CF020E030E054
:106ED00040E050E02AC0B801A701022E04C0769518
:106EE0006795579547950A94D2F781E090E0A0E026
:106EF000B0E004C0880F991FAA1FBB1F2A95D2F7C4
:106F00000197A109B1098E219F21A023B1230097E8
:106F1000A105B10521F081E090E0A0E0B0E09A0188
:106F2000AB01282B392B4A2B5B2BDA01C9018F7758
:106F30009070A070B07080349105A105B10539F44E
:106F400027FF09C0205C3F4F4F4F5F4F04C0215CBB
:106F50003F4F4F4F5F4FE0E0F0E02030A0E03A07B6
:106F6000A0E04A07A0E45A0710F0E1E0F0E0790160
:106F70008A0127C06038710564F5FB01E158FF4FB5
:106F8000D801C7018F779070A070B07080349105E0
:106F9000A105B10539F4E7FE0DC080E490E0A0E062
:106FA000B0E004C08FE390E0A0E0B0E0E80EF91E8E
:106FB0000A1F1B1F17FF05C016950795F794E79446
:106FC000319687E016950795F794E7948A95D1F75F
:106FD00005C0EE24FF248701EFEFF0E06E2F6795E8
:106FE00066276795902F9F77D794DD24D7948E2FAF
:106FF0008695492F462B582F5D29B701CA011F914D
:107000000F91FF90EF90DF900895FC01DB0140812C
:1070100051812281622F6F7770E0221F2227221F69
:107020009381892F880F822B282F30E0991F992771
:10703000991F11969C93119721153105A9F54115BA
:1070400051056105710511F482E037C082E89FEFB8
:1070500013969C938E9312979A01AB0167E0220FCF
:10706000331F441F551F6A95D1F783E08C930DC0E1
:10707000220F331F441F551F12968D919C91139719
:10708000019713969C938E931297203080E03807D7
:1070900080E0480780E4580758F314962D933D93F9
:1070A0004D935C93179708952F3F310579F441155F
:1070B00051056105710519F484E08C93089564FF0E
:1070C00003C081E08C9312C01C9210C02F57304037
:1070D00013963C932E93129783E08C9387E0440F92
:1070E000551F661F771F8A95D1F7706414964D93CC
:1070F0005D936D937C93179708951F93DC01FB01BB
:107100009C91923008F447C08081823008F443C0DB
:10711000943051F411961C91843099F58181682F37
:1071200070E0611B71093FC0843021F0923031F46E
:107130008230B9F18181882389F12DC011961C918B
:1071400011978230F1F081811817D9F412962D91A0
:107150003C911397828193818217930794F02817AB
:107160003907BCF014968D919D910D90BC91A02D86
:107170002481358146815781281739074A075B07E3
:1071800018F4112341F00AC082179307A407B5072A
:1071900040F4112319F061E070E005C06FEF7FEF5C
:1071A00002C060E070E0CB011F910895DC0101C0D6
:1071B0006D9341505040E0F70895AEE0B0E0E3EE4B
:1071C000F8E30C94B43B0D891E8986E08C831A8306
:1071D00009838FEF9FE79E838D83CE014996AC0193
:1071E0006F89788DCE0101960E9400392F813885F4
:1071F000020F131FF80110822E96E4E00C94D03B8E
:10720000ABE0B0E0E6E0F9E30C94A63B3C012B01D7
:107210005A01FC0117821682838181FD03C06FEF42
:107220007FEFC8C19AE0892E1E010894211C311CF1
:10723000F3012381F20123FD859123FF81912F0129
:10724000882309F4B4C1853239F423FD859123FFE5
:1072500081912F01853229F4B30190E00E94F53A23
:10726000E7CF982FDD24CC249924FFE1FD15D0F041
:107270009B3269F09C3228F4903259F0933291F4A9
:107280000EC09D3249F0903369F441E024C052E0D1
:10729000D52A84E0D82A28C098E0D92A25C0E0E180
:1072A000DE2A22C0D7FC29C0892F80538A3070F48F
:1072B000D6FE05C0989C902C1124980E15C0C89C31
:1072C000C02C1124C80EF0E2DF2A0EC09E3229F431
:1072D000D6FC6DC140E4D42A07C09C3619F450E8AE
:1072E000D52A02C0983649F4F20123FD959123FF77
:1072F00091912F01992309F0B8CF892F85548330BC
:1073000018F08052833038F444E050E0A40EB51EEB
:107310005FE359830FC0933631F0933779F093359B
:1073200009F056C020C0F5018081898342E050E019
:10733000A40EB51E710101E010E012C0F501E0805D
:10734000F180D6FC03C06FEF7FEF02C0692D70E0C3
:1073500042E050E0A40EB51EC7010E94EA3A8C013B
:107360005FE7D52214C0F501E080F180D6FC03C0B0
:107370006FEF7FEF02C0692D70E042E050E0A40E95
:10738000B51EC7010E94DF3A8C0150E8D52AD3FE12
:1073900007C01AC0B30180E290E00E94F53ACA9497
:1073A0008C2D90E008171907A8F30EC0F701D7FC41
:1073B0008591D7FE81917F01B30190E00E94F53A5B
:1073C000C110CA94015010400115110579F7ECC0A5
:1073D000943611F0993671F5D7FE08C0F501E080BA
:1073E000F1800281138144E050E00AC0F501808100
:1073F00091817C010027F7FC0095102F42E050E0BE
:10740000A40EB51E5FE6D52217FF0AC010950095A1
:10741000F094E094E11CF11C011D111D80E8D82AB4
:107420002AE030E0A101C801B7010E94213BF82EFB
:10743000F21840C0953729F41D2D1F7E2AE030E058
:107440001DC01D2D197F9F3661F0903720F49835AF
:1074500009F0ADC00FC0903739F0983709F0A7C0D8
:1074600004C028E030E00AC0106114FD146020E17F
:1074700030E004C014FD166020E132E017FF08C0C0
:10748000F501608171818281938144E050E008C000
:10749000F50180819181BC0180E090E042E050E004
:1074A000A40EB51EA1010E94213BF82EF2188FE711
:1074B000D82ED122D6FE0BC05EEFD522F91438F4B7
:1074C000D4FE07C0D2FC05C08FEED82202C01F2D0B
:1074D00001C0192DD4FE0DC0FE01EF0DF11D8081FC
:1074E000803319F499EED92208C01F5FD2FE05C07F
:1074F00003C08D2D867809F01F5F0D2DD3FC14C0BD
:10750000D0FE0FC01C1510F09F2C0BC09F2C9C0CA4
:10751000911A1C2D06C0B30180E290E00E94F53A5A
:107520001F5F1C15C0F304C01C1510F4C11A01C064
:10753000CC2404FF10C0B30180E390E00E94F53A30
:1075400002FF1EC001FD03C088E790E002C088E58D
:1075500090E0B3010CC0802F867891F001FF02C04B
:107560008BE201C080E2D7FC8DE2B30190E00E9483
:10757000F53A06C0B30180E390E00E94F53A9A9490
:10758000F914C0F3FA94F101EF0DF11DB3018081FC
:1075900090E00E94F53AFF20A9F706C0B30180E20F
:1075A00090E00E94F53ACA94CC20C1F741CEF30195
:1075B00066817781CB012B96E2E10C94C23BFC0102
:1075C0000590615070400110D8F7809590958E0F0E
:1075D0009F1F0895FC016150704001900110D8F781
:1075E000809590958E0F9F1F08950F931F93CF93B3
:1075F000DF938C01EB018B8181FF1BC082FF0DC0EB
:107600002E813F818C819D812817390764F4E881A0
:10761000F9810193F983E88306C0E885F985802F15
:107620000995892B31F48E819F8101969F838E83EA
:1076300002C00FEF1FEFC801DF91CF911F910F9193
:107640000895FA01AA27283051F1203181F1E894F8
:107650006F936E7F6E5F7F4F8F4F9F4FAF4FB1E045
:107660003ED0B4E03CD0670F781F891F9A1FA11D40
:10767000680F791F8A1F911DA11D6A0F711D811D41
:10768000911DA11D20D009F468943F912AE0269F06
:1076900011243019305D3193DEF6CF010895462F65
:1076A0004770405D4193B3E00FD0C9F7F6CF462F46
:1076B0004F70405D4A3318F0495D31FD40524193AF
:1076C00002D0A9F7EACFB4E0A6959795879577956C
:1076D0006795BA95C9F700976105710508959B01F3
:1076E000AC010A2E06945795479537952795BA957C
:1076F000C9F7620F731F841F951FA01D089597FB84
:10770000092E07260AD077FD04D00CD006D0002021
:107710001AF4709561957F4F0895F6F790958195CD
:107720009F4F0895AA1BBB1B51E107C0AA1FBB1F97
:10773000A617B70710F0A61BB70B881F991F5A95FD
:10774000A9F780959095BC01CD0108952F923F92A5
:107750004F925F926F927F928F929F92AF92BF9261
:10776000CF92DF92EF92FF920F931F93CF93DF930D
:10777000CDB7DEB7CA1BDB0B0FB6F894DEBF0FBE6A
:10778000CDBF09942A88398848885F846E847D84B7
:107790008C849B84AA84B984C884DF80EE80FD80B9
:1077A0000C811B81AA81B981CE0FD11D0FB6F8942F
:1077B000DEBF0FBECDBFED01089591110EC0803226
:1077C00019F089508550D0F7089591110895815688
:1077D0008A5108F48052855808959927882708957A
:0477E000F894FFCF4B
:1077E40025303458203A09002530325800255820D5
:1077F400000A504553207361797320567070203D00
:107804002025642E25642C50756C73652074696D75
:1078140065203D202564206D73000A5045533A20AD
:1078240025642C25642C25642C25642C25642C25A6
:10783400642C25642C25642C25642C25642C256457
:107844002C2564000A25686400756E6B6E6F776E74
:107854000047414C323256313000000000006901CB
:107864000000000000000000000000000000000014
:10787400000000000800000000000000010048496A
:107884007101041718002C0084002C00C416080091
:107894003D003C003A000A001000DE011400010023
:1078A400020005000A0014001E00280032003C00FB
:1078B400460050005A006400C80000000000B116E1
:1078C400B016B316B216B516B416B716B616B91660
:1078D400B816BB16BA16BD16BC16BF16BE16C11610
:1078E400C016C316C2167479706520253032780A22
:1078F4000025303458203A09000000000000000040
:107904000000010202030303030404040404040446
:107914000405050505050505050505050505050514
:1079240005060606060606060606060606060606F4
:1079340006060606060606060606060606060606E3
:1079440006070707070707070707070707070707C4
:1079540007070707070707070707070707070707B3
:1079640007070707070707070707070707070707A3
:107974000707070707070707070707070707070793
:107984000708080808080808080808080808080874
:107994000808080808080808080808080808080863
:1079A4000808080808080808080808080808080853
:1079B4000808080808080808080808080808080843
:1079C4000808080808080808080808080808080833
:1079D4000808080808080808080808080808080823
:1079E4000808080808080808080808080808080813
:1079F4000808080808080808080808080808080803
:027A0400080078
:00000001FF
